:020000040800F2
:10000000482B0020E101000809460008C934000817
:1000100005460008470300082158000800000000BA
:10002000000000000000000000000000490100087E
:10003000ED030008000000008D010008A551000834
:10004000FB010008FB010008FB010008454D00080A
:10005000FB010008FB010008FB010008FB01000890
:10006000FB010008FB010008FB010008FB01000880
:100070006D0300087D0300088D0300089D03000840
:10008000AD030008BD030008FB010008015800088B
:10009000115800084D0300085D030008FB0100082B
:1000A000FB01000861520008FB010008FB01000889
:1000B0007152000881520008FB010008FB01000892
:1000C000FB010008FB010008FB010008FB01000820
:1000D000FB0100086D5700087D5700088D57000888
:1000E000FB010008FB010008FB010008FB01000800
:1000F000FB010008FB010008FB010008FB010008F0
:10010000FB010008FB010008FB010008FB010008DF
:10011000B1530008C1530008FB010008FB010008AF
:10012000FB010008FB010008CD030008DD03000807
:10013000DFF810D000F0CAF80048004791850008A9
:10014000AFF30080482B0020224B19680868B0E804
:10015000F00F80F30988BFF36F8F4FF0000080F33A
:1001600011884EF00D0E7047000000000648006830
:10017000006880F3088862B661B6BFF34F8FBFF3A3
:100180006F8F00DF00BF00BF08ED00E0EFF30980D4
:10019000BFF36F8F0F4B1A6820E9F00F106008B59E
:1001A0004FF0500080F31188BFF34F8FBFF36F8F74
:1001B00009F0FCF84FF0000080F31188BDE808401A
:1001C00019680868B0E8F00F80F30988BFF36F8FF3
:1001D000704700BFA8010020EFF3058070470000C2
:1001E0000648804706480047FEE7FEE7FEE7FEE7D1
:1001F000FEE7FEE7FEE7FEE7FEE7FEE75F520008E8
:1002000031010008202A04DB203A21FA02F0002103
:10021000704721FA02F3D040C2F120029140084316
:100220001946704740EA01039B0703D009E008C95B
:10023000121F08C0042AFAD203E011F8013B00F8AB
:10024000013B521EF9D27047D2B201E000F8012BF7
:10025000491EFBD270470022F6E710B513460A4646
:1002600004461946FFF7F0FF204610BD30B505469D
:100270002A460B4612F8010B13F8014B08B1A042B5
:10028000F8D01CB1002802D06D1CF1E7284630BD23
:10029000421C10F8011B0029FBD1801A704730B5B1
:1002A0000B46014600202022012409E021FA02F534
:1002B0009D4205D303FA02F5491B04FA02F52844CE
:1002C000151EA2F10102F1DC30BD0000064C074D05
:1002D00006E0E06840F0010394E807009847103416
:1002E000AC42F6D3FFF728FFDCC00008FCC00008D2
:1002F00070B58C1810F8015B15F0070301D110F8E8
:10030000013B2A1106D110F8012B03E010F8016B14
:1003100001F8016B5B1EF9D12B0705D40023521E97
:100320000DD401F8013BFAE710F8013BCB1A921CFF
:1003300003E013F8015B01F8015B521EF9D5A142FD
:10034000D8D3002070BD00BFFEE7000010B5024802
:1003500000F098F910BD0000FC14002010B5024810
:1003600000F090F910BD0000FC14002010B5024808
:1003700000F008FD10BD0000A819002010B50248CB
:1003800000F000FD10BD00006419002010B5024807
:1003900000F0F8FC10BD00009818002010B50248CD
:1003A00000F0F0FC10BD00005418002010B5024809
:1003B00000F0E8FC10BD0000DC18002010B5024879
:1003C00000F0E0FC10BD00002019002010B502482C
:1003D00000F0D8FC10BD0000CC17002010B502487A
:1003E00000F0D0FC10BD0000101800207047000085
:1003F00010B504464FF6FF7322460249024802F048
:10040000F9FF10BDA80A00208817002072B600BFAF
:10041000FEE700000021074AD1610749096941F060
:100420000401054A11611146096941F04001116159
:1004300070470000381A0020002002400021074ABF
:10044000D1610749096941F00201054A116111466C
:100450004861096941F0400111617047381A002074
:10046000002002400022054BDA61054A126942F081
:100470000102034B1A61018070470000381A002006
:100480000020024000201E49C96801F0100139B166
:100490001C49C96941F002011A4AD16140F01000BB
:1004A0001749C96801F0040139B11649C96941F019
:1004B0000101144AD16140F004001149C96901F0F9
:1004C000010169B10F49C96941F004010D4AD161C7
:1004D00000BF0B49C96921F00101094AD16100BF80
:1004E00000BF40F20111884206D10549C96921F0D7
:1004F0000101034AD16101E00149C86000BF7047B2
:1005000000200240381A002070B5044601F0EAF8D5
:10051000054609E0601C38B124B101F0E3F8401B46
:10052000A04201D9032070BD1248C06800F001004C
:100530000028EFD10F48C06800F0200020B100BFB4
:1005400020200C49C86000BF0A48C06800F01000B5
:1005500048B90848C06900F0010020B90548C068E2
:1005600000F0040018B1FFF78DFF0120DBE7002049
:10057000D9E7000000200240F0B504460A46216891
:1005800094F82050012D01D0022D74D1D1F8000231
:1005900040F00100C1F80002107D00F01F060120AC
:1005A00000FA06F3D1F81C029843C1F81C02D06986
:1005B000C8B9D1F80C029843C1F80C02908880B2F7
:1005C000968940EA064601F51070576940F8376091
:1005D000108880B2168940EA064601F51070576906
:1005E00000EBC7004660D069012819D1D1F80C0290
:1005F0001843C1F80C02908880B2168840EA06467B
:1006000001F51070576940F83760908980B21689FB
:1006100040EA064601F51070576900EBC7004660D6
:10062000906928B9D1F804029843C1F8040204E0A3
:10063000D1F804021843C1F80402106928B9D1F8AE
:1006400014029843C1F8140204E0D1F814021843CC
:10065000C1F81402106A012804D1D1F81C02184311
:10066000C1F81C02D1F8000220F00100C1F800021C
:100670000020F0BDFFE7606A40F480206062012046
:10068000F7E770472DE9F05F0446002520684669CA
:100690002068D0F80490206887682068D0F80CA003
:1006A0002068D0F810B02068D0F8188006F001005B
:1006B000002855D007F00100C0B1012021688860F2
:1006C00007F0020018B1204600F057FA0EE007F0DC
:1006D000040010B145F4006508E007F0080010B10F
:1006E00045F4805502E0204600F046FA07F4807099
:1006F000C8B14FF480702168886007F4007018B1A9
:10070000204600F03CFA0EE007F4806010B145F49A
:10071000005508E007F4006010B145F4804502E0A0
:10072000204600F02BFA07F48030C8B14FF4803037
:100730002168886007F4003018B1204600F021FAE3
:100740000EE007F4802010B145F4004508E007F4FE
:10075000002010B145F4803502E0204600F010FA88
:1007600006F0080038B10AF0100020B145F4007519
:1007700010202168C86006F0040040B10AF00800AB
:1007800028B108202168C860204600F0C1F906F0B1
:10079000020038B12068C06800F0030010B12046A4
:1007A00000F0B7F906F0400038B10BF0100020B1AE
:1007B00045F4806510202168086106F0200040B1F2
:1007C0000BF0080028B1082021680861204600F0DD
:1007D000A1F906F0100038B12068006900F00300AC
:1007E00010B1204600F097F906F4003040B109F04E
:1007F000100028B1102021684860204600F08CF9D4
:1008000006F4803040B109F0080028B108202168C2
:100810004860204600F0B6F906F4004088B309F0BD
:10082000040078B306F4807020B108F0010008B12C
:1008300045F0010506F4007020B108F0020008B18F
:1008400045F0020506F4806020B108F0040008B10C
:1008500045F0040506F40060A0B108F0700088B10E
:1008600008F07000402817D006DC10280BD0202894
:100870000CD0302819D10CE0502810D0602814D1A9
:1008800010E01DE019E045F008050FE045F0100507
:100890000CE045F0200509E045F0400506E045F094
:1008A000800503E045F4807500E000BF00BF2068CC
:1008B000806920F070002168886104202168486008
:1008C0002DB1606A284360622046FFF7DAFEBDE87A
:1008D000F09F70B504460CB9012070BD94F820005B
:1008E00010B9204600F0B0F82068006840F0010020
:1008F0002168086000F0F6FE05460DE000F0F2FE0B
:10090000401B0A2808D9606A40F400306062052064
:1009100084F820000120E0E72068406800F0010032
:100920000028EBD02068006820F0020021680860F1
:1009300000F0D8FE05460DE000F0D4FE401B0A286A
:1009400008D9606A40F400306062052084F8200015
:100950000120C2E72068406800F002000028EBD1C7
:10096000207E012806D12068006840F080002168C0
:10097000086005E02068006820F0800021680860B9
:10098000607E012806D12068006840F040002168A0
:10099000086005E02068006820F0400021680860D9
:1009A000A07E012806D12068006840F02000216860
:1009B000086005E02068006820F0200021680860D9
:1009C000E07E012806D12068006820F01000216830
:1009D000086005E02068006840F0100021680860A9
:1009E000207F012806D12068006840F008002168B7
:1009F000086005E02068006820F0080021680860B1
:100A0000607F012806D12068006840F0040021685A
:100A1000086005E02068006820F004002168086094
:100A2000D4E9020108432169084361690843616808
:100A3000491E08432168C86100206062012084F8D3
:100A40002000002049E7000010B586B004460020D1
:100A500002900390049005902A49206888424ED164
:100A600000BF2948C06940F000702749C8610846A6
:100A7000C06900F00070019000BF00BF00BF0846D1
:100A8000806940F0040088610846806900F0040035
:100A9000019000BF00BFC814029000200390049092
:100AA00002A91A4800F066FC4FF480500290022020
:100AB00003900320059002A9144800F05BFC00227B
:100AC0000521132000F0C4FE132000F0B1FE002227
:100AD0000521142000F0BCFE142000F0A9FE002225
:100AE0000521152000F0B4FE152000F0A1FE002223
:100AF0000521162000F0ACFE162000F099FE06B08D
:100B000010BD0000006400400010024000080140D9
:100B10007047704770477047704770B5044694F847
:100B20002000012822D1022084F8200020680068DB
:100B300020F001002168086000F0D4FD05460DE0BA
:100B400000F0D0FD401B0A2808D9606A40F400304C
:100B50006062052084F82000012070BD2068406894
:100B600000F001000028EBD16062F6E7606A40F413
:100B7000002060620120F0E77047704770477047BF
:100B80007047704770470146002291F82100022803
:100B900008D00420886300BF002081F8200000BF37
:100BA000012070470868006820F00E000B6818608C
:100BB0000868006820F001000B68186091F8403068
:100BC00001209840CB6B5860012081F8210000BFC4
:100BD000002081F8200000BF1046E2E770B504460F
:100BE000002594F82100022803D00420A0630125E9
:100BF000C1E02068006820F00E00216808602068CD
:100C0000006820F00100216808605C492068884283
:100C100052D95A4978392068884201D1012047E0E9
:100C2000564964392068884201D1102040E0534978
:100C300050392068884201D1801539E04F493C394C
:100C40002068884201D1801432E04C49283920685C
:100C5000884202D14FF480302AE048491439206894
:100C6000884202D14FF4801022E044492068884233
:100C700001D140041CE042492068884201D1012092
:100C800016E03F4914312068884201D110200FE05E
:100C90003B4928312068884201D1801508E0384955
:100CA0003C312068884201D1801401E04FF480304B
:100CB0003349091F086051E030497839206888427B
:100CC00001D1012047E02D4964392068884201D1D3
:100CD000102040E0294950392068884201D1801510
:100CE00039E026493C392068884201D1801432E03D
:100CF000224928392068884202D14FF480302AE006
:100D00001E4914392068884202D14FF4801022E035
:100D10001A492068884201D140041CE01849206823
:100D2000884201D1012016E015491431206888421B
:100D300001D110200FE0124928312068884201D1EA
:100D4000801508E00E493C312068884201D18014AA
:100D500001E04FF48030094980394860012084F86F
:100D6000210000BF002084F8200000BF606B10B19C
:100D70002046616B8847284670BD00008000024015
:100D80000804024070B50446E06B056820680668F8
:100D900094F84010042088402840002875D006F0C0
:100DA00004000028FAD02068006800F0200028B96C
:100DB0002068006820F0040021680860D549206898
:100DC000884254D9D34978392068884201D1042017
:100DD00049E0D04964392068884201D1402042E08E
:100DE000CC4950392068884201D100153BE0C949FF
:100DF0003C392068884202D14FF4804033E0C54935
:100E000028392068884202D14FF480202BE0C14964
:100E100014392068884202D14FF4800023E0BD4994
:100E20002068884201D1C0041DE0BB492068884287
:100E300001D1042017E0B84914312068884201D15B
:100E4000402010E0B44928312068884201D10015C3
:100E500009E0B1493C312068884202D14FF480401A
:100E600001E04FF48020AC49091F086054E0A94913
:100E700078392068884201D104204AE0A5496439C4
:100E80002068884202D1402043E04CE0A14950391B
:100E90002068884201D100153BE09E493C3920681A
:100EA000884202D14FF4804033E09A4928392068C3
:100EB000884202D14FF480202BE0964914392068F3
:100EC000884202D14FF4800023E092492068884292
:100ED00001D1C0041DE090492068884201D104205E
:100EE00017E08D4914312068884201D1402010E07C
:100EF000894928312068884201D1001509E08649D6
:100F00003C312068884202D14FF4804001E04FF428
:100F10008020804980394860E06A002802D020465D
:100F2000E16A8847F4E094F84010022088402840A5
:100F3000002871D006F002000028FAD0206800686E
:100F400000F0200040B92068006820F00A00216805
:100F50000860012084F821006E492068884254D935
:100F60006C4978392068884201D1022049E06949FA
:100F700064392068884201D1202042E06549503917
:100F80002068884201D140153BE062493C39206825
:100F9000884202D14FF4005033E05E49283920687E
:100FA000884202D14FF400302BE05A4914392068AE
:100FB000884202D14FF4001023E05649206888424D
:100FC00001D180041DE054492068884201D10220EB
:100FD00017E0514914312068884201D1202010E0E7
:100FE0004D4928312068884201D1401509E04A491D
:100FF0003C312068884202D14FF4005001E04FF4A8
:1010000000304549091F086054E04249783920689A
:10101000884202D102204AE057E03E496439206804
:10102000884201D1202042E03A4950392068884264
:1010300001D140153BE037493C392068884202D154
:101040004FF4005033E0334928392068884202D1F8
:101050004FF400302BE02F4914392068884202D128
:101060004FF4001023E02B492068884201D180040E
:101070001DE029492068884201D1022017E0264955
:1010800014312068884201D1202010E02249283103
:101090002068884201D1401509E01F493C31206891
:1010A000884202D14FF4005001E04FF4003019495A
:1010B0008039486000BF002084F8200000BFA06A8B
:1010C00030B32046A16A884722E094F840100820F7
:1010D00088402840E0B106F00800C8B120680068E8
:1010E00020F00E002168086094F84010012088402C
:1010F000E16B48600120A06384F8210000BF00205C
:1011000084F8200000BF206B10B12046216B884777
:1011100070BD000080000240080402400146002229
:1011200009B9012070471E4B086898420BD21D4B2D
:101130000868C01A1423B0FBF3F080000864194853
:101140000838C8630AE0164B0868C01A1423B0FBBD
:10115000F3F08000086412480838C863022081F860
:1011600021000868026843F6F0708243D1E9010368
:101170001843CB6818430B6918434B6918438B69B4
:101180001843CB6918430243086802600020886353
:10119000012081F82100002081F8200000BFC1E774
:1011A000080402400800024070B5044600F09AFAB4
:1011B00006462546681C10B104480078054400BF67
:1011C00000F090FA801BA842FAD370BDA001002065
:1011D0002DE9F04104460E460127002500BF2648B0
:1011E000007E012802D10220BDE8F08101202249C1
:1011F000087600BF2068022813D14CF25030FFF768
:1012000083F990BB0120FFF705F94CF25030FFF74E
:101210007BF907461948006920F004001749086166
:1012200023E04CF25030FFF76FF9F0B94FF0FF3088
:101230003060A56812E02846FFF700F94CF2503004
:10124000FFF762F907460D48006920F002000B49DC
:1012500008610FB1356007E005F50065D4E90210BB
:1012600001EBC020A842E6D800BF00BF0020024921
:10127000087600BF3846B7E7381A00200020024041
:101280000348006940F08000014908610020704770
:10129000002002402DE9FE4F05468B461746984632
:1012A000012600240020029000BF2448007E01286F
:1012B00002D10220BDE8FE8F01202049087600BF40
:1012C0004CF25030FFF720F9064686BB012D02D1C3
:1012D0000120029006E0022D02D10220029001E0DE
:1012E0000420029000241EE02201B946C24648466E
:1012F0005146FEF787FF80B20190022000FB04B048
:1013000000900199FFF7AEF84CF25030FFF7FCF86F
:1013100006460B48006920F001000949086106B142
:1013200004E0601CC4B202988442DDDB00BF00BF51
:1013300000200249087600BF3046BBE7381A00207B
:101340000020024000200849096901F0800151B1E4
:101350000649054A5160064951601146096901F084
:10136000800101B101207047002002402301674540
:10137000AB89EFCD2DE9F847024600239C467BE17F
:101380004FF0010808FA03F4D1F8008008EA0400DD
:10139000A0427DD1DFF8F4A2D1F80480A8EB0A09BD
:1013A000D0453AD014DCB8F1030F50D009DCB8F1C5
:1013B000000F31D0B8F1010F1CD0B8F1020F49D1A4
:1013C00020E0B8F1110F18D0B8F1120F42D11EE091
:1013D000B9F5881F25D006DCB9F5803F20D0B9F5D6
:1013E000801F37D11AE0B9F5001F18D0B9F5041FD6
:1013F00030D117E0D1F80CC02DE0D1F80C8008F105
:10140000040C28E0D1F80C8008F1080C23E0D1F896
:101410000C8008F10C0C1EE000BF00BF00BF00BF35
:1014200000BF00BFD1F80880B8F1000F02D14FF023
:10143000040C0BE0D1F80880B8F1010F03D14FF094
:10144000080C146102E04FF0080C546103E04FF007
:10145000000C00E000BF00BFFF2801D8904601E06B
:1014600002F104084646FF2802D84FEA830803E049
:10147000A3F108084FEA88084746D6F800804FF0E5
:101480000F0909FA07F928EA09080CFA07F900E038
:101490007AE048EA0908C6F80080D1F8048008F02C
:1014A0008058B8F1805F6FD100BFDFF8E481D8F8D1
:1014B000188048F00108DFF8D891C9F81880C846AC
:1014C000D8F8188008F00108CDF8008000BF00BFF0
:1014D0004FEAB9384FEA930958F829504FEA837810
:1014E0004FEA18794FF00F0808FA09F825EA0805BD
:1014F000DFF8A081424502D14FF0000824E0DFF878
:101500009881424502D14FF001081DE0DFF88C813F
:10151000424502D14FF0020816E0DFF884814245CF
:1015200002D14FF003080FE0DFF87881424502D185
:101530004FF0040808E0DFF87081424502D14FF017
:10154000050801E04FF006084FEA83794FEA197960
:1015500008FA09F848EA0505DFF850814FEA9309CF
:1015600048F82950D1F8048008F48038B8F5803F55
:101570000BD1DFF83C81D8F8008048EA0008DFF89A
:101580003091C9F800800AE075E0DFF82481D8F8CE
:10159000008028EA0008DFF81891C9F80080D1F827
:1015A000048008F40038B8F5003F0ED1DFF8008160
:1015B00008F10408D8F8008048EA0008DFF8F09045
:1015C00009F10409C9F800800DE0DFF8E48008F1B2
:1015D0000408D8F8008028EA0008DFF8D49009F160
:1015E0000409C9F80080D1F8048008F48018B8F51F
:1015F000801F0ED1DFF8B88008F10808D8F8008005
:1016000048EA0008DFF8A89009F10809C9F8008045
:101610000DE0DFF89C8008F10808D8F8008028EA7F
:101620000008DFF88C9009F10809C9F80080D1F8AA
:10163000048008F40018B8F5001F0ED1DFF87080A0
:1016400008F10C08D8F8008048EA0008DFF860903C
:1016500009F10C09C9F800800DE0DFF8548008F1A9
:101660000C08D8F8008028EA0008DFF8449009F157
:101670000C09C9F800805B1CD1F8008028FA03F837
:10168000B8F1000F7FF47CAEBDE8F88700001110C0
:101690000010024000080140000C01400010014011
:1016A0000014014000180140001C014008000140E6
:1016B00000040140024693680B400BB1012000E09A
:1016C0000020704710B5C26821EA020302EA010453
:1016D00043EA0443036110BD0AB1016101E00B0458
:1016E00003617047014800687047000098010020BE
:1016F00003480068034909780844014908607047B5
:1017000098010020A001002010B50848006840F0B2
:10171000100006490860032000F0D8F80F2000F000
:1017200007F800F055F8002010BD0000002002402E
:10173000F0B587B0044600260027002500BF1F48EB
:10174000806940F400601D4988610846806900F4A2
:101750000060009000BF00BF01A902A800F0C8FA15
:1017600000F0FEFA06461648B6FBF0F0471E154894
:101770001549086040F2E7311348C1604760002115
:1017800001618160816101F075F8054695B90E48E7
:1017900001F0E0F805466DB9192000F049F8102C69
:1017A00007D200222146192000F052F807480460B1
:1017B00000E00125284607B0F0BD000000100240FF
:1017C00040420F00002C0140EC1900209C01002039
:1017D00008B500BF1448806940F0010012498861D3
:1017E0000846806900F00100009000BF00BF00BF04
:1017F0000846C06940F08050C8610846C06900F0E2
:101800008050009000BF00BF00220F21901E00F00A
:101810001FF800BF0549486820F0E06040F0007004
:10182000486000BF08BD00000010024000000140F9
:1018300001460846002809DB00F01F0301229A40F8
:1018400043099B0003F1E023C3F8002100BF704768
:101850002DE9F05F80460D461646002704F00CF88F
:10186000074639462A46334601F00700C0F1070A09
:10187000BAF1040F02D94FF0040A01E0C0F1070ADF
:10188000D14600F1040ABAF1070F02D24FF0000A64
:1018900001E0A0F1030AD4464FF0010A0AFA09FA5E
:1018A000AAF1010A0AEA020A0AFA0CFA4FF0010B3D
:1018B0000BFA0CFBABF1010B0BEA030B4AEA0B042E
:1018C0002146404603F0E0FFBDE8F09F00BF00F076
:1018D0000702064B19684FF6FF031940044B0B43F0
:1018E00043EA0221014B196000BF70470CED00E094
:1018F0000000FA05012001490862704700000E420D
:101900002DE9F04385B0064642A30FCB01AC0FC4CE
:1019100044A0006800904FF0000800250027002434
:10192000A146042E36D004DC012E3BD0022E6BD112
:101930005FE0082E32D0102E66D13B484468006824
:1019400000F0807000B301A8C4F38341475C04F445
:10195000803070B134484068C0F340401DF80080CA
:1019600004F4803040B13148B0FBF8F000FB07F5DB
:1019700002E02F4807FB00F52B48406800F4800088
:10198000B0F5800F01D1A94603E068000321B0FB48
:10199000F1F93AE000F0F4F9814636E000F0F0F9B0
:1019A000814632E02048046A04F44070B0F5807F3C
:1019B00005D104F0020010B14FF4004918E004F41E
:1019C0004070B0F5007F07D11748406A00F0020070
:1019D00010B149F640490BE004F44070B0F5407F87
:1019E00006D11148006800F4003008B14FF22449D4
:1019F0000BE000F0B5F90C494968C1F38131491C8D
:101A00004900B0FBF1F900E000BF00BF484605B057
:101A1000BDE8F08302030405060708090A0B0C0D54
:101A20000E0F1010010200000010024000127A0098
:101A300000093D00F8B5044600260025207800F096
:101A4000010000286BD000274348C06900F0805097
:101A500070B900BF4048C06940F080503E49C8613D
:101A60000846C06900F08050009000BF00BF012709
:101A70003A48006800F48070B0B93848006840F413
:101A8000807036490860FFF72DFE064606E0FFF736
:101A900029FE801B642801D90320F8BD2F48006867
:101AA00000F480700028F2D02B48006A00F44075E2
:101AB0002DB3A08800F44070A84220D02648006AC8
:101AC00020F4407501202649086000200860224863
:101AD000056205F0010090B1FFF704FE064608E03C
:101AE000FFF700FE801B41F28831884201D90320B4
:101AF000D3E71948006A00F002000028F0D0164829
:101B0000006A20F440706168084313490862012F9D
:101B100004D10846C06920F08050C86100BF207819
:101B200000F00200022807D10B48406820F4404032
:101B3000A168084308494860207800F01000102888
:101B400007D10548406820F48000616908430249D4
:101B500048600020A1E70000001002400070004033
:101B60004004424270B504460D460CB9012070BDD8
:101B70005A48006800F00700A8420ED25748006893
:101B800020F007002843554908600846006800F027
:101B90000700A84201D00120E9E7207800F0020008
:101BA00002281DD1207800F00400042805D14C48FB
:101BB000406840F4E0604A494860207800F008003E
:101BC000082805D14648406840F4605044494860C0
:101BD0004348406820F0F000A1680843404948604D
:101BE000207800F0010078B36068012806D13C48F5
:101BF000006800F4003090B90120B8E7606802285E
:101C000006D13748006800F0007040B90120AEE707
:101C10003348006800F0020008B90120A7E7304807
:101C2000406820F00300616808432D494860FFF7D1
:101C300059FD064609E0FFF755FD801B41F288314A
:101C4000884202D9032092E707E02548406800F067
:101C50000C006168B0EB810FEDD12048006800F006
:101C60000700A8420ED91D48006820F0070028434D
:101C70001A4908600846006800F00700A84201D031
:101C8000012074E7207800F00400042807D11448EC
:101C9000406820F4E060E16808431149486020781A
:101CA00000F00800082808D10D48406820F4605072
:101CB000216940EAC1000A49486000F061F808491A
:101CC0004968C1F30311074A515CC84006490860DE
:101CD00006480068FFF72CFD002048E7002002407E
:101CE0000010024094C00008A40100209C010020C4
:101CF0000F2202600D4A526802F0030242600B4A52
:101D0000526802F0F0028260084A526802F4E0620F
:101D1000C260064A526802F46052D2080261044A64
:101D2000126802F007020A607047000000100240CB
:101D3000002002400148006870470000A401002014
:101D400000B5FFF7F7FF04494968C1F30221034AD0
:101D5000515CC84000BD000000100240A4C0000853
:101D600000B5FFF7E7FF04494968C1F3C221034A00
:101D7000515CC84000BD000000100240A4C0000833
:101D8000F0B585B00FF26C0C9CE8E01001A8A0E85B
:101D9000E0101CA52D6800950021002200230024DE
:101DA0000020194D696801F00C05F5B1042D02D031
:101DB000082D19D101E0154819E001ADC1F38346A2
:101DC000AC5D01F4803555B10F4D6D68C5F34045EC
:101DD0001DF805200D4D6543B5FBF2F302E00C4DF7
:101DE00004FB05F3184602E000BF084800BF00BF2F
:101DF00005B0F0BD02030405060708090A0B0C0D27
:101E00000E0F1010010200000010024000127A00B4
:101E100000093D00F8B504460CB90120F8BD207852
:101E200000F00100002878D0F848406800F00C006D
:101E300004280CD0F548406800F00C00082811D1A7
:101E4000F248406800F48030B0F5803F0AD1EF4896
:101E5000006800F4003000285FD0606800285CD182
:101E60000120DBE700BF6068B0F5803F06D1E7489E
:101E7000006840F48030E549086028E0606858B99F
:101E8000E248006820F48030E049086008460068B5
:101E900020F4802008601AE06068B0F5A02F0BD114
:101EA000DA48006840F48020D84908600846006895
:101EB00040F4803008600AE0D448006820F48030A4
:101EC000D24908600846006820F48020086000BFFE
:101ED000606888B1FFF706FC054606E0FFF702FCE4
:101EE000401B642801D9032098E7C848006800F423
:101EF00000300028F2D010E0FFF7F4FB054606E0C2
:101F0000FFF7F0FB401B642801D9032086E7BF4898
:101F1000006800F400300028F2D1207800F00200C0
:101F2000022857D1B948406800F00C0050B1B748BA
:101F3000406800F00C00082818D1B448406800F44C
:101F4000803098B9B148006800F0020020B12069E3
:101F5000012801D0012061E7AC48006820F0F800BA
:101F6000616940EAC100A949086033E02069E8B12D
:101F70000120A7490860FFF7B5FB054606E0FFF71B
:101F8000B1FB401B022801D9032047E79F480068A6
:101F900000F002000028F2D09C48006820F0F80011
:101FA000616940EAC1009949086013E0002098493E
:101FB0000860FFF797FB054606E0FFF793FB401B21
:101FC000022801D9032029E79048006800F00200A8
:101FD0000028F2D1207800F0080008282DD1A0694F
:101FE000B8B101208B490860FFF77CFB054606E08D
:101FF000FFF778FB401B022801D903200EE7834836
:10200000406A00F002000028F2D0012002F040FEF9
:1020100013E000207F490860FFF764FB054606E0F7
:10202000FFF760FB401B022801D90320F6E6774842
:10203000406A00F002000028F2D1207800F004008D
:10204000042873D100277148C06900F0805070B92E
:1020500000BF6E48C06940F080506C49C8610846B6
:10206000C06900F08050009000BF00BF01276A489F
:10207000006800F48070B0B96748006840F4807070
:1020800065490860FFF72EFB054606E0FFF72AFBCF
:10209000401B642801D90320C0E65F48006800F4B3
:1020A00080700028F2D000BFE068012806D15748B0
:1020B000006A40F001005549086227E0E06858B91D
:1020C0005248006A20F00100504908620846006A40
:1020D00020F00400086219E0E06805280BD14B48A5
:1020E000006A40F00400494908620846006A40F06E
:1020F000010008620AE04548006A20F001004349F7
:1021000008620846006A20F00400086200BFE06828
:10211000A0B1FFF7E7FA054609E0FFF7E3FA401B35
:1021200041F28831884202D9032077E622E037481D
:10213000006A00F002000028EFD012E0FFF7D2FAA8
:10214000054608E0FFF7CEFA401B41F2883188428D
:1021500001D9032062E62D48006A00F00200002841
:10216000F0D1012F05D12948C06920F080502749BE
:10217000C86100BFE069C8B32448406800F00C00A3
:10218000082860D0E069022848D10020204908666C
:10219000FFF7A8FA054606E0FFF7A4FA401B02285D
:1021A00001D903203AE61948006800F000700028C1
:1021B000F2D1206AB0F5803F07D11448406820F47E
:1021C0000030A168084311494860D4E90801084378
:1021D0000E49496821F4741108430C4948600120F4
:1021E0000B490866FFF77EFA054607E03DE0FFF77A
:1021F00079FA401B022801D903200FE60348006842
:1022000000F000700028F2D02FE000000010024023
:102210000000424280044242007000400020144905
:102220000866FFF75FFA054606E0FFF75BFA401B1A
:10223000022801D90320F1E50E48006800F0007083
:102240000028F2D111E0E069012800D1E6E5094853
:10225000466806F48031206A814204D106F4701188
:10226000606A814201D00120D8E50020D6E5000057
:10227000000042420010024010B503460022002038
:10228000024A02EB81021468A0B210BD006C00404B
:1022900010B503460020034800EB810094B20460AF
:1022A00010BD0000006C00407047704710B5044638
:1022B0002068006800F00100F0B12068406800F07C
:1022C0000100C8B120684068C0F3800048B12046D2
:1022D000FFF7EBFF6FF00400216848600420607492
:1022E00004E02046FFF7E0FF0120607420684068AA
:1022F00020F001002168486010BD000070B5044660
:1023000000250CB9012070BD607C20B9002020742C
:10231000204600F05BF802206074204600F068F967
:1023200018B1042060740120EDE7204602F0CFFCD4
:1023300018B1042060740120E5E72068406820F0AF
:10234000070021684860A06828B11F48006820F095
:1023500001001D4908601C48001F006820F46070DF
:10236000A16808431849091F08606068401C08B14B
:10237000656809E00120FFF7C3FA05461DB904208E
:1023800060740120BFE76D1E2068806820F00F0098
:1023900040EA1540216888602068C06865F30F0036
:1023A0002168C860204602F0AFFC18B104206074B8
:1023B0000120A8E70021E17301216173A1730120CD
:1023C000607400209FE70000306C004038B5044680
:1023D0000F49206888421AD1FFF78CFA00BF0D48D8
:1023E000C06940F000600B49C8610846C06900F050
:1023F0000060009000BF00BF012007490860002274
:1024000005210320FFF724FA0320FFF711FA38BD56
:1024100000280040001002403C0442422DE9F047F1
:1024200004460D46904600260027B14604B115B972
:102430000120BDE8F08700BF207C012801D10220E7
:10244000F7E70120207400BF02206074B8F1000F8C
:1024500006D1E978E17369786173A978A1730BE01B
:10246000E87802F029FCE073687802F025FC6073DC
:10247000A87802F021FCA073A27B617BE07B02F0D4
:102480008FFC2073207B2870204602F06FFC0646EC
:102490004FF46160B6FBF0F9B9F1180F2FD918208D
:1024A000B9FBF0F000EB4000C000C0EB4011C1EB05
:1024B0000020A6EB00163146204602F0CAFC38B1D7
:1024C0000420607400BF0020207400BF0120B0E72A
:1024D000204602F03FFC0746781C80B1B7420ED27E
:1024E0000B4807443946204602F09CFC38B10420D2
:1024F000607400BF0020207400BF012099E7012014
:10250000607400BF0020207400BF00BF91E700008E
:10251000805101002DE9F04704460D469046002603
:10252000002704B115B90120BDE8F08700BF207C69
:10253000012801D10220F7E70120207400BF02200A
:102540006074B8F1000F0BD128784FF461614843F3
:102550006978C1EB011100EB8100A978461812E0FF
:10256000287802F0A9FB4FF4616100FB01F968785B
:1025700002F0A2FBC0EB001009EB8009A87802F082
:102580009BFB09EB00063146204602F062FC38B1A5
:102590000420607400BF0020207400BF0120C3E746
:1025A0002068406820F0050021684860204602F05D
:1025B000D1FB0746781C80B1B7420ED20B480744C6
:1025C0003946204602F02EFC38B10420607400BF6A
:1025D0000020207400BF0120A6E70120607400BF26
:1025E0000020207400BF00BF9EE700008051010062
:1025F00070B5044600250CB9012070BD2068406804
:1026000020F0080021684860FFF76CF8054607E0F5
:10261000FFF768F8401BB0F57A7F01D90320ECE79B
:102620002068406800F008000028F1D00020E4E7AE
:1026300010B504460CB9012010BD606A38B9606855
:10264000B0F5827F00D105E00021E16102E00021C8
:10265000216161610021A16294F8510028B9002034
:1026600084F85000204600F043F8022084F851001E
:102670002068006820F0400021680860A08800F40D
:102680008270218901F404410843A18901F40061A9
:102690000843217C01F002010843217D01F0010182
:1026A0000843218B01F400710843217F01F03801B8
:1026B00008432021095D01F080010843218D01F4C8
:1026C00000510843216808600421A06901EA104014
:1026D000216848602068C06920F400602168C861F2
:1026E00000206065012084F851000020A4E700006C
:1026F00010B586B004460020029003900490059027
:102700002F492068884225D100BF2E48806940F4B7
:1027100080502C4988610846806900F480500190FF
:1027200000BF00BF00BF0846806940F00400886118
:102730000846806900F00400019000BF00BFA0209F
:102740000290022003900320059002A91E48FEF784
:1027500011FE33E01D49206888422FD100BF19487F
:10276000C06940F480401749C8610846C06900F458
:102770008040019000BF00BF00BF0846806940F064
:10278000080088610846806900F00800019000BFD9
:1027900000BF4FF4204002900220039003200590D8
:1027A00002A90B48FEF7E6FD4FF48040029000209E
:1027B0000390049002A90648FEF7DCFD06B010BDA8
:1027C0000030014000100240000801400038004085
:1027D000000C01407047704730B502460B4600BF01
:1027E00092F83C00012801D1022030BD012082F87E
:1027F0003C0000BF022082F83D0010684468106869
:10280000816824F070041868044310684460144D13
:102810001068A84213D0134D1068A8420FD010685A
:10282000B0F1804F0BD0104D1068A84207D00F4D6B
:102830001068A84203D00E4D1068A84205D121F0BF
:1028400080015868014310688160012082F83D00D2
:1028500000BF002082F83C0000BF00BFC5E70000B9
:10286000002C0140003401400004004000080040FA
:10287000000C004010B504460CB9012010BD94F8BE
:102880003D0028B9002084F83C00204600F026F8DE
:10289000022084F83D00211D206802F0FFFC012089
:1028A00084F8460000BF84F83E0001213F20015516
:1028B000402001554120015500BF00BF012084F890
:1028C000420043200155442001554520015500BFD9
:1028D000012084F83D000020D0E7000038B5044610
:1028E0002068B0F1804F16D100BF1848C06940F091
:1028F00001001649C8610846C06900F00100009057
:1029000000BF00BF002205211C20FEF7A1FF1C20F4
:10291000FEF78EFF19E00E492068884215D100BFEE
:102920000A48C06940F002000849C8610846C06909
:1029300000F00200009000BF00BF002205211D2012
:10294000FEF786FF1D20FEF773FF38BD0010024022
:1029500000040040014691F83D00012801D001200B
:102960007047022081F83D000868C06840F001000F
:102970000B68D860164B0868984213D0154B08684E
:1029800098420FD00868B0F1804F0BD0124B086806
:10299000984207D0114B0868984203D0104B086842
:1029A00098420CD10868806800F00702062A0CD013
:1029B0000868006840F001000B68186005E00868CE
:1029C000006840F001000B6818600020C8E70000B4
:1029D000002C014000340140000400400008004089
:1029E000000C00402DE9F04104460D4600BF94F86C
:1029F0003C00012802D10220BDE8F081012084F8CA
:102A00003C0000BF022084F83D002068866826F064
:102A1000770626F47F46206886602868502833D0E1
:102A20000CDC202850D004DC00284BD0102851D1D9
:102A300049E0302849D040284CD139E060282DD0D9
:102A4000702807D0B0F5805F03D0B0F5005F41D1AA
:102A50000DE040E0D5E902136A68206802F06CFCE2
:102A60002068866846F077062068866033E0D5E9FE
:102A700002136A68206802F05FFC2068806840F4F6
:102A800080402168886026E0EA686968206802F072
:102A900067FC5021206802F05AFC1CE0EA68696873
:102AA000206802F070FC6021206802F050FC12E007
:102AB000EA686968206802F053FC4021206802F04F
:102AC00046FC08E000BF00BF00BF2968206802F094
:102AD0003EFC00E000BF00BF012084F83D0000BFC5
:102AE000002084F83C0000BF00BF85E7704710B5A8
:102AF000044620680069C0F34000D8B12068C0686F
:102B0000C0F34000B0B16FF00200216808610120FD
:102B100020772068806900F0030018B12046FFF795
:102B2000E5FF05E0204600F0ADF8204600F0ABF8E8
:102B30000020207720680069C0F38000D8B12068A9
:102B4000C068C0F38000B0B16FF004002168086174
:102B5000022020772068806900F4407018B1204678
:102B6000FFF7C4FF05E0204600F08CF8204600F097
:102B70008AF80020207720680069C0F3C000D8B12F
:102B80002068C068C0F3C000B0B16FF008002168D1
:102B90000861042020772068C06900F0030018B1A4
:102BA0002046FFF7A3FF05E0204600F06BF8204623
:102BB00000F069F80020207720680069C0F3001059
:102BC000D8B12068C068C0F30010B0B16FF0100039
:102BD00021680861082020772068C06900F44070EF
:102BE00018B12046FFF782FF05E0204600F04AF8C2
:102BF000204600F048F8002020772068006900F0A7
:102C0000010058B12068C06800F0010030B16FF0D9
:102C1000010021680861204600F036F8206800694C
:102C2000C0F3C01058B12068C068C0F3C01030B104
:102C30006FF08000216808612046FFF7CBFD206817
:102C40000069C0F3801058B12068C068C0F38010DC
:102C500030B16FF0400021680861204600F02EF886
:102C600020680069C0F3401058B12068C068C0F304
:102C7000401030B16FF02000216808612046FFF756
:102C8000AAFD10BD7047704710B50446084920687A
:102C9000884201D1FEF72CFD00BF06480068B0F164
:102CA000804F03D101210448FEF70CFD00BF10BD89
:102CB000002C0140E81500200010014070477047CB
:102CC000704700002DE9F84F044620680568206829
:102CD000C668206847694FF00009CA4605F00F0929
:102CE000B9F1000F0AD105F0200038B106F020003C
:102CF00020B1204602F0E3FBBDE8F88FB9F1000FE8
:102D000071D007F0010018B906F4907000286AD05D
:102D100005F0010030B106F4807018B1206C40F06D
:102D20000100206405F0040030B107F0010018B183
:102D3000206C40F00200206405F0020030B107F082
:102D4000010018B1206C40F00400206405F0080078
:102D500048B106F0200010B907F0010018B1206C4E
:102D600040F008002064206C68B305F0200028B112
:102D700006F0200010B1204602F0A1FB2068406957
:102D8000C0F3801A206C00F0080010B9BAF1000FEF
:102D900022D0204602F068FB2068406900F0400025
:102DA000B0B12068406920F0400021684861A06B04
:102DB00050B15648A16B4863A06BFDF70FFF10B1EF
:102DC000A06B416B88470CE02046FFF779FF08E0D5
:102DD0002046FFF775FF04E02046FFF771FF002053
:102DE000206489E7FFE7206B012878D105F0100007
:102DF000002874D006F01000002870D000BF00201A
:102E0000009020680068009020684068009000BF33
:102E100000BF2068406900F04000C0B3A06B0068AC
:102E200040681FFA80F8B8F1000F2FD0A08D404500
:102E30002CDDA4F82E80A06B806920281FD020688C
:102E4000C06820F480702168C8602068406920F064
:102E50000100216848612068406920F04000216835
:102E60004861202084F83E00002020632068C0686C
:102E700020F010002168C860A06BFDF784FEA08DD3
:102E8000E28D801A81B22046FFF719FF34E7FFE791
:102E9000A08DE18D401A1FFA80F8E08DE8B1B8F1FD
:102EA000000F1AD02068C06820F490702168C860B4
:102EB0002068406920F0010021684861202084F8E2
:102EC0003E00002020632068C06820F010002168C8
:102ED000C86041462046FFF7F2FE0DE7FFE705F028
:102EE000800030B106F0800018B1204602F0D8FB17
:102EF00002E705F0400030B106F0400018B120466E
:102F000002F0CDFAF8E600BFF6E6000055540008DE
:102F100010B504460CB9012010BDA06900B100E055
:102F200000BF94F83D0028B9002084F83C002046FA
:102F300000F028F8242084F83D002068C06820F4C0
:102F400000502168C860204602F02CFB2068006910
:102F500020F49040216808612068406920F02A0030
:102F6000216848612068C06840F400502168C8604A
:102F700000202064202084F83D0084F83E000020DA
:102F8000CAE7000010B586B0044600200290039006
:102F900004900590FE49206888426AD100BFFD4830
:102FA000C06940F40020FB49C8610846C06900F4CC
:102FB0000020019000BF00BF00BF0846806940F0BC
:102FC000100088610846806900F01000019000BF81
:102FD00000BF08150290022003900320059002A96B
:102FE000ED48FEF7C7F94FF400600290002003900F
:102FF000049002A9E848FEF7BDF9E848E8490860EE
:10300000002048600021E64881608021C1600021E5
:10301000016141618161C161FEF780F808B1FDF78E
:10302000F5F900BFDE48A063446200BFDB482830EA
:10303000DC490860102048600021DA488160802166
:10304000C1600021016141618161C161FEF766F8E3
:1030500008B1FDF7DBF900BFD2486063446200BFEE
:10306000002205213420FEF7F3FB3420FEF7E0FBBD
:10307000BDE1CD492068884243D100BFC548C06941
:1030800040F48010C349C8610846C06900F480104C
:10309000019000BF00BF00BF0846806940F01000EB
:1030A00088610846806900F01000019000BF00BFF1
:1030B00000BF0846806940F02000886108468069AA
:1030C00000F02000019000BF00BF88140290022091
:1030D00003900320059002A9AF48FEF74BF90420A6
:1030E000029000200390049002A9B048FEF742F934
:1030F000002205213520FEF7ABFB3520FEF798FBBB
:1031000075E1AB49206888426AD100BFA148806957
:1031100040F480409F4988610846806900F48040FF
:10312000019000BF00BF00BF0846806940F0040066
:1031300088610846806900F00400019000BF00BF6C
:1031400048150290022003900320059002A9994897
:10315000FEF710F94FF48060029000200390049075
:1031600002A99448FEF706F99348944908600020A4
:1031700048600021914881608021C1600021016187
:1031800041618161C161FDF7C9FF08B1FDF73EF9F9
:1031900000BF8A48A063446200BF8748143888494A
:1031A0000860102048600021854881608021C1604E
:1031B0000021016141618161C161FDF7AFFF08B18B
:1031C000FDF724F900BF7E486063446200BF00221F
:1031D00005212520FEF73CFB2520FEF729FB06E113
:1031E0007849206888426AD100BF6A48C06940F4C3
:1031F00000306849C8610846C06900F40030019099
:1032000000BF00BF00BF0846806940F0040088612D
:103210000846806900F00400019000BF00BF042050
:103220000290022003900320059002A96148FEF756
:10323000A1F80820029000200390049002A95D48A4
:10324000FEF798F85C4814305F4908600020486039
:1032500000215D4881608021C160002101614161E0
:103260008161C161FDF75AFF08B1FDF7CFF800BFDA
:103270005548A063446200BF4F4828305349086056
:10328000102048600021514881608021C1600021E8
:10329000016141618161C161FDF740FF08B1FDF746
:1032A000B5F800BF49486063446200BF00220521B1
:1032B0002620FEF7CDFA2620FEF7BAFA97E0444919
:1032C000206888428BD100BF3248C06940F480201A
:1032D0003049C8610846C06900F48020019000BFF1
:1032E00000BF00BF0846806940F0080088610846BA
:1032F000806900F00800019000BF00BF081502902F
:10330000022003900320059002A93248FEF732F80C
:103310004FF40060029000200390049002A92D4811
:10332000FEF728F8244828382B4908600020486018
:103330000021294881608021C16000210161416133
:103340008161C161FDF7EAFE08B1FDF75FF800BFDA
:103350002148A063446200BF17483C381F490860F9
:103360001020486000211D4881608021C16000213B
:10337000016141618161C161FDF7D0FE08B1FDF7D6
:1033800045F800BF15486063446200BF002227E093
:10339000004C004000100240001001403004024088
:1033A000CC170020101800200050004000140140ED
:1033B0000038014000080140580002405418002025
:1033C0009818002000440040DC180020201900203C
:1033D00000480040000C014064190020A81900209A
:1033E00005212720FEF734FA2720FEF721FA06B040
:1033F00010BD70472DE9F84F04460E461746994612
:103400004FF0000A94F83D0020285AD106B117B9B0
:103410000120BDE8F88F00BF94F83C00012801D1DD
:103420000220F6E7012084F83C0000BF0020206461
:10343000212084F83D00FEF755F98246A784E784F1
:10344000A068B0F5805F04D1206910B90025B046AE
:1034500002E035464FF0000800BF002084F83C0031
:1034600000BF1BE05346002280212046CDF800908B
:1034700002F046F908B10320CBE745B9B8F80000DF
:10348000C0F308002168486008F1020803E02878CA
:10349000216848606D1CE08C401EE084E08C0028B0
:1034A000E0D15346002240212046CDF8009002F0A2
:1034B00027F908B10320ACE7202084F83D00002064
:1034C000A7E70220A5E7704700BFFEE710B5082177
:1034D0003C48FEF7EFF83C490870084600783B4945
:1034E0000978884208D03848007838490870FEF7D3
:1034F000F9F83749086062E0FEF7F4F834490968E2
:10350000401A32285BD930480078002853D131481E
:10351000007800284DD1304800780C2845D2DFE8EB
:1035200000F006121F44444444203132333400BFBB
:1035300000202949087048708870C8700120274908
:10354000087000BF31E000BF0120234908704870B7
:10355000002088700120C8702049087000BF24E056
:1035600000BF1D484078042808D01B484078401C04
:103570001949487008468078401E88700120174914
:10358000087012E000BF00BF00BF00BF1248007803
:103590001149087001204870002088700320C8700D
:1035A00001200E49087000BF00BF00BF012009497B
:1035B0000870012010BD002006490870FAE70020BD
:1035C000F8E70000000C01404C0100204D010020F4
:1035D00050010020440100200C020020F0000020D7
:1035E00010B510213C48FEF765F83C4908700846C4
:1035F00000783B490978884208D038480078384933
:103600000870FEF76FF83749086062E0FEF76AF865
:1036100034490968401A32285BD9304800780028BC
:1036200053D13148007800284DD1304800780C281B
:1036300045D2DFE800F006121F44444444203132F2
:10364000333400BF00202949087048708870C87062
:1036500001202749087000BF31E000BF0120234945
:1036600008700020487001208870C87020490870D8
:1036700000BF24E000BF1D488078032808D01B4805
:103680004078401E1949487008468078401C887070
:1036900001201749087012E000BF00BF00BF00BF43
:1036A0001248007811490870002048700120887085
:1036B0000320C87001200E49087000BF00BF00BF82
:1036C000012009490870012010BD0020064908703A
:1036D000FAE70020F8E70000000C01405401002048
:1036E0005501002058010020450100200C02002057
:1036F000F00000201CB520216D48FDF7DBFF6D496F
:103700000870084600786C490978884208D06948F2
:10371000007869490870FDF7E5FF68490860C5E071
:10372000FDF7E0FF65490968401A3228F7D961487A
:103730000078002870D16248007800286DD1614877
:1037400000780C2813D2DFE800F0061334469A9A6A
:103750009A55696A6B6C00BF01205A49087048701D
:10376000002088700120C8705749087000BF86E0AB
:103770005448407801280DD100BF022051490870FB
:1037800004204870002088700220C87001204E4933
:1037900008700DE000BF07204A49087004204870F7
:1037A000002088700220C87001204749087000BFBF
:1037B00065E000BF43484078C0F107004149087008
:1037C00004204870002088700320C87001203E4902
:1037D000087000BF53E000BF03203A49087004207E
:1037E0004870002088700420C87001203649087095
:1037F00000BF44E000BF33484078C0F10C003149BD
:10380000087001204870002088700320C8700120D3
:103810002D49087000BF32E044E041E000BF00BF26
:1038200000BF28484078012814D100BF25480078FF
:103830002449087001204870002088700420C87056
:1038400001202149087000BF20480068401C1F4922
:10385000086013E000BF1B4800781A490870002078
:103860004870012088700420C87001201649087033
:1038700000BF16480068401C1449086000BF00BF24
:103880001048C0780F498978CDE900100D48437879
:1038900002780FA10FA001F0DFFF01200849087096
:1038A00001201CBD002006490870FAE70020F8E757
:1038B000000C01405C0100205D010020600100203F
:1038C000460100200C020020F00000209806002095
:1038D0004B3300002D2D2D3E2573207072657373C0
:1038E000656409256420202025642020202564208B
:1038F000202025640A00000010B540213C48FDF757
:10390000D9FE3C490870084600783B49097888424E
:1039100008D03848007838490870FDF7E3FE374989
:10392000086062E0FDF7DEFE34490968401A32287B
:103930005BD930480078002853D1314800780028FE
:103940004DD1304800780C2845D2DFE800F044061D
:103950001220212223133233343500BF002029499D
:10396000087048708870C87001202749087000BF2F
:1039700031E000BF00BF01202249087048700020DC
:1039800088700120C8702049087000BF23E000BF84
:1039900000BF00BF00BF02201A4908700420487011
:1039A000002088700220C87001201749087000BFED
:1039B00011E000BF00BF00BF00BF07201149087021
:1039C00004204870002088700220C87001200E4931
:1039D000087000BF00BF00BF012009490870012026
:1039E00010BD002006490870FAE70020F8E7000043
:1039F000000C0140640100206501002068010020E6
:103A0000470100200C020020F000002010B50AA0A1
:103A100001F022FF00224FF400410A48FDF75CFE4E
:103A20004FF47A60FDF7C0FB0020074908700120C1
:103A30000649087010BD00004274207265736574F9
:103A40000D0A0000000801406F0100206E010020F7
:103A500010B501209B49087000209B498860012017
:103A60009A4908609A48486001200873994805F00F
:103A7000C7F999490880084600884FF6FF718842C7
:103A80001CD101231A4695A195A005F0BDF930B1CE
:103A9000904801F0C7FE96A001F0DEFE17E001237A
:103AA0001A468EA196A005F0AFF918B198A001F0C2
:103AB000D3FE0CE09BA001F0CFFE08E08648008812
:103AC0004AF6AA21884202D199A001F0C5FE9C487D
:103AD0000078052820D2DFE800F003306291C000B2
:103AE00001231A4697A19CA005F08EF9A8B10020E9
:103AF0007449087001209B4908709B490870012394
:103B00001A4676A199A005F07FF910B19BA001F0AB
:103B1000A3FE9EA001F0A0FED2E001231A469FA1C1
:103B20008DA005F071F910B19EA001F095FE8448BA
:103B30000078401C8249087000BF9EA001F08CFEF6
:103B400089480078002829D101231A469DA1A0A008
:103B500005F05AF978B101231A4660A19FA005F03B
:103B600053F9D8B1A1A001F077FE75480078401C48
:103B70007349087012E001231A46A0A194A005F031
:103B800043F940B1A0A001F067FE6D480078401CE9
:103B90006B49087002E0FFF739FF91E000BF7248FF
:103BA0000078002829D101231A469DA19FA005F085
:103BB0002BF978B101231A4648A19FA005F024F9FA
:103BC000D8B1A1A001F048FE5D480078401C5C49D6
:103BD000087012E001231A469FA194A005F014F981
:103BE00040B1A0A001F038FE55480078401C54496F
:103BF000087002E0FFF70AFF62E000BF5A48007851
:103C0000002829D101231A469CA19FA005F0FCF8A9
:103C100078B101231A4631A19EA005F0F5F8D8B17C
:103C2000A0A001F019FE46480078401C44490870E5
:103C300012E001231A469FA193A005F0E5F840B1D8
:103C40009FA001F009FE3E480078401C3C490870E6
:103C500002E0FFF7DBFE33E000BF434800780028B6
:103C60002ED103231A469CA1A2A005F0CDF898B14D
:103C700000201449087001203A49087001231A46AF
:103C800016A13AA005F0C0F810B13CA001F0E4FD87
:103C90009EA001F0E1FD13E0052303229EA195A063
:103CA00005F0B2F828B1A1A001F0D6FDFFF7AEFEF5
:103CB00006E0A149A1A001F0CFFDFFF7A7FE00BFDC
:103CC00000BF10BDF10000200C020020980600206B
:103CD0003175746400500708720100204F4B0000DA
:103CE00041542B52455345543D310D0A000000000C
:103CF000B8B4CEBBC9E8B1B8B3C9B9A60D0A0000C3
:103D000041542B444953434F4E4E3D300D0A000061
:103D1000C8A1CFFBC1ACBDD3CBF9D3D0C9E8B1B8F2
:103D20000D0A0000B8B4CEBBCAA7B0DC0D0A000073
:103D3000B7C7CAD7B4CEC6F4B6AF0D0A00000000AC
:103D40006F0100202B4445563A302C313031303051
:103D5000303030303030330041542B4445563F0D25
:103D60000A0000006C0100206D01002041542B412D
:103D700055544F5F4346473D310D0A00D7D4B6AF87
:103D8000D6D8C1ACB4F2BFAA0D0A0000C9E8B1B8D8
:103D9000D2D1C1ACBDD30D0A000000002B44455662
:103DA0003A000000CEB4C1ACBDD3C9E8B1B80D0A29
:103DB00000000000C9E8B1B8CEB4C1ACBDD30D0A53
:103DC000000000002B55554944533A464646300002
:103DD00041542B55554944533F0D0A0041542B552E
:103DE000554944533D303030320D0A00C9E8D6C33E
:103DF000D6F7B7FECEF1B3C9B9A60A002B5555497F
:103E000044533A30303032005555494453B7C7C453
:103E1000ACC8CFD6B5A3ACB7FBBACF0A0000000040
:103E20002B555549444E3A464646310041542B5590
:103E30005549444E3F0D0A0041542B555549444EB7
:103E40003D464630340D0A00C9E8D6C3B6C1B7FEB8
:103E5000CEF1B3C9B9A60A002B555549444E3A468E
:103E600046303400555549444EB7C7C4ACC8CFD6C8
:103E7000B5A3ACB7FBBACF0A000000002B555549DB
:103E800044573A464646320041542B55554944570B
:103E90003F0D0A0041542B55554944573D4646466F
:103EA000350D0A00C9E8D6C3D0B4B7FECEF1B3C908
:103EB000B9A60A002B55554944573A46464635009F
:103EC0005555494457B7C7C4ACC8CFD6B5A3ACB74E
:103ED000FBBACF0A000000002B434F4E4E4543541F
:103EE00045443A302C3130313030303030303030A1
:103EF0003300000041542B434F4E4E3D31303130A2
:103F000030303030303030330D0A0000C1ACBDD31A
:103F1000B3C9B9A6A3A100002B434F4E4E4543544D
:103F20002054494D454F555400000000C1ACBDD34D
:103F3000B3ACCAB1A3A10000A80A0020C1ACBDD394
:103F4000CAA7B0DCA3A120257300000000B58BB088
:103F500019481A4908600420486000211748816008
:103F6000C1604FF4A02101614FF480114161002133
:103F7000017641768176C17601774177FCF7A9FC1D
:103F800008B1FCF743FA0020069007900120089042
:103F90000020019002900390049005900120099068
:103FA0000E200A9001A90548FCF7E6FA0348FCF741
:103FB000B4FD0BB000BD000000640040FC14002004
:103FC00008B500BF2D48406940F001002B49486109
:103FD0000846406900F00100009000BF00BF00BF2C
:103FE0000846406940F0020048610846406900F018
:103FF0000200009000BF00BF002205210C20FDF749
:1040000027FC0C20FDF714FC002205210D20FDF7F4
:104010001FFC0D20FDF70CFC002205210E20FDF7F2
:1040200017FC0E20FDF704FC002205210F20FDF7F0
:104030000FFC0F20FDF7FCFB002205211020FDF7EF
:1040400007FC1020FDF7F4FB002205211120FDF7ED
:10405000FFFB1120FDF7ECFB002205213A20FDF7C4
:10406000F7FB3A20FDF7E4FB002205213B20FDF79A
:10407000EFFB3B20FDF7DCFB08BD00000010024019
:1040800000B59DB01C22184916A8FCF7CBF80021FA
:1040900016A804F09AFB154908601C2212491C312D
:1040A0000FA8FCF7BFF800210FA804F08EFB104901
:1040B00008601C220C49383108A8FCF7B3F800212D
:1040C00008A804F082FB0B4908601C220649543101
:1040D00001A8FCF7A7F8002101A804F076FB064927
:1040E00008601DB000BD000024C00008840100204D
:1040F000880100208C0100209001002000B585B0CF
:104100000020019002900390049000BF3D48806918
:1041100040F010003B4988610846806900F01000BB
:10412000009000BF00BF00BF0846806940F020003B
:1041300088610846806900F02000009000BF00BF41
:1041400000BF0846806940F0040088610846806925
:1041500000F00400009000BF00BF00BF0846806967
:1041600040F0080088610846806900F0080000906F
:1041700000BF00BF002240F211212348FDF7ACFA36
:10418000012248F212012148FDF7A6FA002240213F
:104190001E48FDF7A1FA012280211B48FDF79CFA79
:1041A00040F2912001900120029000200390022013
:1041B000049001A91448FDF7DDF848F2420001908F
:1041C00001200290002003900220049001A90F48D2
:1041D000FDF7D0F8102001900120029000200390FC
:1041E0000320049001A90948FDF7C4F87820019044
:1041F000002002900120039001A90548FDF7BAF8BC
:1042000005B000BD00100240001001400008014050
:10421000000C01401FB500200290019000BF5648DD
:10422000C06940F000605449C8610846C06900F0A8
:104230000060009000BF00BF00BF0846C06940F0AA
:104240008050C8610846C06900F08050009000BFEF
:1042500000BF4A484A4908604FF0FF3048600021DB
:1042600047488160FEF74AF808B1FCF7CFF8012112
:104270004348FEF701F845F2510188424CD0132023
:104280008DF8080000208DF809008DF80A00012241
:1042900002A93B48FEF73EF908B1FCF7B7F8042045
:1042A0008DF8040001208DF8050018208DF8060017
:1042B00023208DF80700012201A93148FEF7AEF84E
:1042C00008B1FCF7A3F82E480068006840F0010030
:1042D0002B49096808600198039045F251020121B9
:1042E0002748FDF7D5FF9DF80F2002212448FDF750
:1042F000CFFF9DF80D2003212148FDF7C9FF9DF850
:104300000E2004211E48FDF7C3FF9DF80C20052157
:104310001B48FDF7BDFF2DE002211948FDF7ACFF5A
:10432000C0B28DF80F0003211548FDF7A5FFC0B2FC
:104330008DF80D0004211248FDF79EFFC0B28DF8E4
:104340000E0005210E48FDF797FFC0B28DF80C0056
:1043500003980190002201A90948FEF75FF808B10F
:10436000FCF754F806480068006840F00100044972
:10437000096808601FBD00000010024000280040CE
:104380002415002010B50F480F4908604FF48270C3
:1043900048604FF400410C4881600021C160016118
:1043A00041614FF4007181610821C1610021016206
:1043B000416281620A21C162FEF73AF908B1FCF755
:1043C00025F810BD003001403815002010B50E480A
:1043D0000E4908604FF48270486000210B488160EC
:1043E000C160016141614FF4007181610021C161CF
:1043F0000162416281620A21C162FEF719F908B1C6
:10440000FCF704F810BD00000038004090150020B3
:1044100000B587B0002003900490059006900190AD
:1044200002904FF080401449086009204860002144
:104430001148816041F63F71C160002101618161D5
:10444000FEF718FA08B1FBF7E1FF4FF48050039034
:1044500003A90948FEF7C6FA08B1FBF7D7FF002009
:104460000190029001A90448FEF7B6F908B1FBF7E4
:10447000CDFF07B000BD0000E815002000B587B0F3
:10448000002003900490059006900190029015483A
:104490001549086041F28730486000211248816068
:1044A00041F63F71C160002101618161FEF7E2F9CF
:1044B00008B1FBF7ABFF4FF48050039003A90A4803
:1044C000FEF790FA08B1FBF7A1FF002001900290DF
:1044D00001A90548FEF780F908B1FBF797FF07B07F
:1044E00000BD0000000400403016002010B50B484D
:1044F0000B4908604FF4E1304860002108488160B2
:10450000C16001610C21416100218161C161FEF73F
:10451000FFFC08B1FBF77AFF10BD0000004C004023
:104520007816002010B50B480B4908604FF4E130B5
:104530004860002108488160C16001610C2141612F
:1045400000218161C161FEF7E3FC08B1FBF75EFF6A
:1045500010BD000000500040BC16002010B50B48F4
:104560000B4908604FF4E130486000210848816041
:10457000C16001610C21416100218161C161FEF7CF
:10458000C7FC08B1FBF742FF10BD00000038014036
:104590000017002010B50B480B4908604FF4E130BC
:1045A0004860002108488160C16001610C214161BF
:1045B00000218161C161FEF7ABFC08B1FBF726FF6A
:1045C00010BD0000004400404417002010B50B4807
:1045D0000B4908604FF4E1304860002108488160D1
:1045E000C16001610C21416100218161C161FEF75F
:1045F0008FFC08B1FBF70AFF10BD00000048004027
:104600008817002000BFFEE700BFFEE770B500245A
:104610000CE0002506E00020074901EBC501085524
:10462000681CC5B2802DF6DB601CC4B2082CF0DB20
:1046300000F0F0F870BD00001802002010B504462C
:104640001CB90021A62000F0E1FA012C03D10021C1
:10465000A72000F0DBFA10BD10B504463CB90021DC
:10466000C82000F0D3FA0021A12000F0CFFA012CDD
:1046700007D10021C02000F0C9FA0021A02000F0DD
:10468000C5FA10BDF0B514460B46CF1701EB5777AE
:10469000C7F3C702CF1701EB5777FF10A1EBC7078E
:1046A000FEB20123B340DDB24CB1134B03EBC003A8
:1046B0009B5C2B43104F07EBC007BB541AE00E4B1B
:1046C00003EBC0039B5CDB430B4F07EBC007BB5402
:1046D000094B03EBC0039B5C2B43074F07EBC00761
:1046E000BB54054B03EBC0039B5CDB43024F07EB62
:1046F000C007BB54F0BD0000180200201FB5A02069
:10470000009001200190039069464048FCF732FE7A
:104710000122A0213D48FCF7DFFF002210213C4888
:10472000FCF7DAFFC820FCF73FFD012210213848D2
:10473000FCF7D2FF0021AE2000F068FA0021022031
:1047400000F064FA0021102000F060FA00214020FF
:1047500000F05CFA0021B02000F058FA002181201E
:1047600000F054FA0021CF2000F050FA0021A120DF
:1047700000F04CFA0021A62000F048FA0021A82001
:1047800000F044FA00213F2000F040FA0021AD2063
:1047900000F03CFA00218B2000F038FA0021332091
:1047A00000F034FA0021C82000F030FA0021D320B4
:1047B00000F02CFA0021084600F028FA0021D5204C
:1047C00000F024FA0021802000F020FA0021D920F6
:1047D00000F01CFA00211F2000F018FA0021DA2056
:1047E00000F014FA0021122000F010FA0021DB2062
:1047F00000F00CFA0021402000F008FAFFF706FF55
:104800000021AF2000F002FA1FBD000000080140A7
:104810000010014070B500241CE004F1B001C8B2E2
:10482000002100F0F3F90021022000F0EFF900214F
:10483000102000F0EBF9002508E0084901EBC50164
:10484000085D012100F0E2F9681CC5B2802DF4DB9F
:10485000601CC4B2082CE0DB70BD00001802002010
:104860002DE9FE4F0746884692461C460197CDF833
:104870000080082C02D14FF006091FE02046E31704
:1048800004EB5373DB1021464FEAE47C04EB5C7CC1
:104890004FEAEC0CA4EBCC0CBCF1000F02D04FF0B3
:1048A000010C01E04FF0000C6344224604EBD27C83
:1048B0004FEA6C0C03FB0CF303F0FF09AAF1200094
:1048C000C6B200255EE0082C07D106EB46002F4952
:1048D00001EB400010F805B01DE00C2C07D106EBF1
:1048E00046002B4901EB800010F805B013E0102CB6
:1048F00005D1284800EB061010F805B00BE0182C85
:1049000007D106EBC600244901EB800010F805B082
:1049100001E0BDE8FE8F002002901CE00BF00100DA
:1049200028B1414638460C9AFFF7ACFE09E00C98D6
:1049300008B9012000E00020024641463846FFF752
:10494000A1FE4FEA6B0B08F1010000F0FF0802988E
:10495000401CC0B2029002980828DFDB781CC7B266
:10496000082C0BD004EBD4714A100199791A8A42B1
:1049700004D1019F00980830C0B20090DDF800809B
:10498000681CC5B24D459EDB00BFC2E7049A000813
:104990002C9C0008A0A0000890A600082DE9FC4F60
:1049A0000746884616461C46BB46CDF8048020467E
:1049B000E21704EB5272D2102146E31704EB537353
:1049C000DB10A4EBC3030BB1012300E000231A4466
:1049D000624392B20092002575E0102C05D13C484C
:1049E00000EB461010F805903BE0182C07D106EBC1
:1049F000C600384901EBC00010F8059031E0202CCA
:104A000005D1354800EBC61010F8059029E0402C80
:104A100005D1324800EB462010F8059021E00C2C1F
:104A200007D106EB46002E4901EBC00010F80590B7
:104A300017E00E2C07D1C6EBC6002A4901EB800017
:104A400010F805900DE0122C09D106EBC60000EB22
:104A50004000254901EB400010F8059001E0BDE859
:104A6000FC8F4FF0000A1CE009F0010028B141461C
:104A700038460B9AFFF706FE09E00B9808B90120AB
:104A800000E00020024641463846FFF7FBFD4FEAB2
:104A9000690908F1010000F0FF080AF1010000F0C7
:104AA000FF0ABAF1080FDFDB781CC7B2A7EB0B00D7
:104AB000A04204D15F4601980830C0B20190DDF8F1
:104AC0000480681C85B20098854286DB00BFC6E77B
:104AD000ECB30008ACB70008F4B7000874B80008DD
:104AE00074BA00080CBC000874BE00082DE9FF4F22
:104AF00005460E4617461C46DDF838904FF0000A72
:104B00000095B3462046E21704EB5272D2102146BC
:104B1000E31704EB5373DB10A4EBC3030BB10123C6
:104B200000E000231A44D4B24FF0000845E0002012
:104B300003903BE00D9810F80A0002900AF1010082
:104B40001FFA80FA002001901DE0029800F0010099
:104B500028B14A4631462846FFF794FD0AE0B9F1EC
:104B6000000F01D1012000E0002002463146284616
:104B7000FFF788FD029840100290701CC6B20198A1
:104B8000401CC0B2019001980828DEDB681CC5B249
:104B90000098281AB84204D1009D0BF1080000F0DB
:104BA000FF0B5E460398401CC0B203900398B842C6
:104BB000C0DB08F1010000F0FF08A045B7DBBDE84D
:104BC000FF8F2DE9F84106460F4614461D46DDF8D5
:104BD0001C8013E0CDF8008022782B463946304601
:104BE000FFF73EFE082D02D1B01DC6B205E02846F3
:104BF00005EBD07106EB6101CEB2641C2078202851
:104C000002DB20787E28E5DDBDE8F88170B504463A
:104C10000E462EB1012240211C48FCF75DFD04E048
:104C2000002240211948FCF757FD002210211748A7
:104C3000FCF752FD00251BE0002220211348FCF761
:104C40004BFD04F0800028B1012280210F48FCF7C1
:104C500043FD04E0002280210C48FCF73DFD0122C9
:104C600020210A48FCF738FD6006040E681CC5B216
:104C7000082DE1DB012210210448FCF72DFD012263
:104C800040210248FCF728FD70BD000000080140EB
:104C900008B508490968C9084FF47A72B1FBF2F106
:104CA0004143009100BF00BF00994A1E00920029B5
:104CB000F9D108BDA4010020014600BF080900EB9E
:104CC0008000420001F00F001044C0B2704770B580
:104CD00004460025FCF706FD054607E0FCF702FD4B
:104CE000401BB0F57A7F01D9032070BD2068406871
:104CF00000F020000028F1D02068406840F010004B
:104D0000216848600020F0E770B50446002520685F
:104D1000406820F0100021684860FCF7E3FC05467D
:104D200007E0FCF7DFFC401BB0F57A7F01D90320D8
:104D300070BD2068406800F020000028F1D00020FD
:104D4000F6E7000010B50248FDF7B0FA10BD00000C
:104D5000241500200146002200230868006A82B260
:104D60000868406A83B243EA0240704730B50146A2
:104D700000220023002400200D68AD69AAB20D684E
:104D8000ED69ACB20D68AD69ABB29A4205D00D6861
:104D9000ED6963F31F45284601E044EA024030BD57
:104DA000F0B504460B460021002504F5FA61032BFB
:104DB0001BD2C3EBC30000EB03100926B0FBF6F0D7
:104DC0001044001D4618481E06EB90066427B0FBF1
:104DD000F7F0361A481EBF00B0FBF7F03044072644
:104DE000B0FBF6F706FB17051AE0C3EBC30000EBB8
:104DF00003100926B0FBF6F01044001D084400EB38
:104E000091006426B1FBF6F6801B4FF4C876B1FB27
:104E1000F6F63044801E0726B0FBF6F706FB1705B2
:104E2000E8B2F0BD70B504460D4600262046FFF7F7
:104E30004EFF08B101260AE0280C21680862A8B2DA
:104E4000216848622046FFF75FFF00B10126304627
:104E500070BD70B504460D4600262046FFF737FFAB
:104E600008B101260AE0280C21688861A8B22168EF
:104E7000C8612046FFF748FF00B10126304670BDEB
:104E800008B501201023504A022100901420FFF79A
:104E900098FE01200E231022022100903720FFF7F8
:104EA0007DFD01200E231122022100904B20FFF7EF
:104EB00075FD01201023454A112100901420FFF7B1
:104EC00080FE01200E231022112100903720FFF7D1
:104ED00065FD01200E231122114600904B20FFF7A3
:104EE0005DFD012010233A4A202100901420FFF795
:104EF00068FE01200E231022202100903720FFF7AA
:104F00004DFD01200E231122202100904B20FFF7A0
:104F100045FD012010232F4A2F2100901420FFF778
:104F200050FE01200E2310222F2100903720FFF782
:104F300035FD01200E2311222F2100904B20FFF779
:104F40002DFD2548407804280BD12348807840B9AE
:104F500000201023214A022100906420FFF731FE37
:104F600031E01D48407803280CD11B488078012887
:104F700008D100201023194A112100906420FFF766
:104F800020FE20E01448407802280CD11248807896
:104F9000022808D100201023104A2021009064200C
:104FA000FFF70FFE0FE00C48407801280BD10A48AC
:104FB0008078032807D100201023084A2F21009071
:104FC0006420FFF7FEFD08BD070100200B01002053
:104FD0000F010020130100200C020020000100201E
:104FE0001F48007801280BD11E48007840B91E48A0
:104FF0000078662804D14FF470401C4988602DE089
:105000001748007860B917480078012808D1164879
:105010000078662804D14FF48050144988601DE060
:105020001048007858B90E48007840B90E4800780A
:10503000662804D14FF480500C4988600EE009487E
:10504000007801280AD10648007838B90648007867
:10505000662803D14FF480500449886070470000EF
:105060007E0100207F010020A80A00200C02002001
:1050700010B51C48C078042833D11A480078082895
:105080000BD018480078092807D0164800780A285D
:1050900003D0144800780B2823D112484078012807
:1050A0000ED111480FC800F075FD4FF47A70FCF76F
:1050B0007BF800200B49087001200C49087010E0B3
:1050C0000848407868B908480FC803F023FB4FF43C
:1050D0007A70FCF769F80020024908700120034942
:1050E000087010BD0C02002098060020F00000207F
:1050F00000BF012003F058FBFFF772FFFFF7B8FF76
:10510000F7E7000000BF012003F04EFB00BF03F0F3
:10511000AFFF084807C800F085FDFFF77BFB00BF25
:1051200004F00AFA044800780028ECD0FEF790FC5E
:10513000E9E700000C0200206E01002000BF012002
:1051400003F032FBFBE7000000BF4FF47A7003F07E
:105150002BFB0E4800780028F7D00D48007848B99E
:105160000C48007830B90C48007818B90B48007822
:105170000028EAD00A480078082803DB08480078AD
:105180000B28E2DD03F0EEF9DFE700006C01002000
:10519000390100203A0100203B0100203C010020A1
:1051A0000C02002010B500BF502080F31188BFF31F
:1051B0004F8FBFF36F8F00BF04F0F2FA18B14FF0BA
:1051C00080500449086000BF002080F3118800BFB0
:1051D00010BD000004ED00E000B595B028210BA83B
:1051E000FBF739F8142106A8FBF735F818216846B3
:1051F000FBF731F809200B904FF480300C90002021
:105200000D9001200F90119002201290C103139174
:105210004FF4E01114910BA8FCF7FCFD08B1FBF76B
:10522000F5F80F20069002200790002008904FF418
:105230008060099000200A90022106A8FCF792FCE9
:1052400008B1FBF7E3F801200090400201906846A6
:10525000FCF7F0FB08B1FBF7D9F815B000BD7047BB
:1052600010B50248FDF743FC10BD0000EC1900200A
:1052700010B50248FDF73BFC10BD0000E81500200A
:1052800010B54FF400710348FCF71CFA0248FDF713
:105290002EFC10BD001001403016002010B5026831
:1052A000204B98420ED0204B98420BD0B0F1804F4B
:1052B00008D01E4B984205D01D4B984202D01D4B82
:1052C000984203D122F070024B681A43154B984262
:1052D0000ED0154B98420BD0B0F1804F08D0134B35
:1052E000984205D0124B984202D0124B984203D1FB
:1052F00022F44072CB681A4322F080034C6943EADF
:10530000040202608B68C3620B688362054B98429B
:1053100002D0054B984201D10B690363012343611D
:1053200010BD0000002C014000340140000400408A
:1053300000080040000C004030B50C46816821F4A4
:105340007F4142EA032525432943816030BD0A4657
:10535000816821F0700142F00703194381607047B2
:1053600030B50B461446026A056A25F00105056250
:10537000816921F0F00141EA041122F00A021A4386
:105380008161026230BD30B50B461446056A25F0D6
:10539000100505628169026A21F4704141EA043115
:1053A00022F0A00242EA03128161026230BD0000D5
:1053B00010B50248FDF786FC10BD000078160020ED
:1053C00010B51F480068002808DD1E480068006806
:1053D000C0F3001010B10020194908601948006896
:1053E0000068C0F3401030B3164800684068C4B28B
:1053F00015481349096844541148006840F2FF31C8
:10540000884204D20E480068401C0D4908600C48D0
:1054100000880E4908800A4801680D48FAF71BFF0A
:10542000002004E00849095C094A1154401C044961
:1054300009688842F6DB0348FDF744FC10BD000014
:1054400094010020BC160020A80600207001002056
:10545000A80A002070B505466C6A0020E085E0844B
:105460002046FDF72DFC70BD0168C96821F49071DC
:105470000268D1600168496921F001010268516147
:10548000016B012905D10168C96821F0100102688A
:10549000D160202180F83E1000210163704710B5D3
:1054A00004462068C06820F040002168C8602020C1
:1054B00084F83D002046FEF706F8002010BDF8B540
:1054C000044694F83E00222869D1A068B0F5805FB8
:1054D0000CD1206950B90025A66A20684068C0F345
:1054E00008003080A06A801CA06215E0A56A002632
:1054F000A068B0F5805F03D0A06828B9206918B90A
:1055000020684068287004E02068406800F07F0050
:105510002870A06A401CA062E08D401E80B2E08529
:10552000A8BB2068C06820F020002168C8602068FF
:10553000C06820F480702168C8602068406920F04D
:10554000010021684861202084F83E00206B01287A
:105550001ED1002020632068C06820F01000216860
:10556000C8602068006800F0100010280AD100BF51
:10557000002000902068006800902068406800903B
:1055800000BF00BFA18D2046FDF799FB03E004E0BA
:105590002046FDF72EFF0020F8BD0020FCE702208A
:1055A000FAE7000070B504462168096921F440510A
:1055B000E2681143226811612269A168114362699E
:1055C00041EA02052168C96841F20C62914329430E
:1055D0002268D1602168496921F44071A2691143B0
:1055E000226851612D4A2168914202D1FCF7B8FB33
:1055F00001E0FCF7A5FB00EBC00101EB00116268C4
:105600009200B1FBF2F100EBC00202EB0012636802
:105610009B00B2FBF3F26423B2FBF3F202EBC20392
:1056200003EB0212A1EB8201322202EB0111642290
:10563000B1FBF2F101F0F00100EBC00202EB00124D
:1056400063689B00B2FBF3F26423B2FBF3F201EB5D
:10565000021200EBC00101EB001163689B00B1FB7B
:10566000F3F100EBC00303EB00136668B600B3FB75
:10567000F6F36426B3FBF6F303EBC30606EB031362
:10568000A1EB8301322303EB01116423B1FBF3F19E
:1056900001F00F0111442268916070BD0038014093
:1056A000014691F83D00212828D18868B0F5805F37
:1056B0000BD1086948B90A6A1088C0F308000B6862
:1056C0005860086A801C086205E00B6A581C086272
:1056D00018780B685860C88C401E80B2C88458B9CE
:1056E0000868C06820F080000B68D8600868C0684F
:1056F00040F040000B68D860002070470220FCE7B3
:105700002DE9F04104460D4617469846069E21E0D5
:10571000701CF8B12EB1FBF7E5FFA0EB0800B0421A
:1057200018D92068C06820F4D0702168C86020684B
:10573000406920F0010021684861202084F83D0084
:1057400084F83E0000BF002084F83C0000BF032026
:10575000BDE8F081206800682840A84201D10120FE
:1057600000E00020B842D3D00020F1E710B5024895
:10577000FDF7A8FA10BD00000017002010B5024880
:10578000FDF7A0FA10BD00004417002010B5024834
:10579000FDF798FA10BD00008817002070B5054687
:1057A0000E461446A2B24FF6FF7331462846FDF767
:1057B00021FEA2B24FF6FF7331460248FDF71AFEF2
:1057C00070BD00008817002070B505460C462046C5
:1057D000FAF75EFD86B24FF6FF7332462146284641
:1057E000FDF708FE2046FAF753FD86B24FF6FF7329
:1057F000324621460148FDF7FDFD70BD88170020A7
:1058000010B50248FAF73EFF10BD0000FC1400205E
:1058100010B50248FAF736FF10BD0000FC14002056
:1058200000BFFEE770B504460025204600F0E2F90F
:10583000FBF788FD0748844209D14AF6AA252A4683
:10584000002321460120FBF725FD064600BFFBF79C
:1058500017FD70BD005007080FB4054B10B503A924
:10586000044A029800F034F810BC5DF814FB000004
:10587000CD5C00080802002002480068C0F3022046
:10588000704700000CED00E010B5002804DB0A07AB
:10589000130E054A135406E00A07140E034A00F0DB
:1058A0000F031B1FD45410BD00E400E018ED00E00E
:1058B00002E008C8121F08C1002AFAD170477047D9
:1058C000002001E001C1121F002AFBD17047000037
:1058D0002DE9FF4F8BB09A460F460546002606E09D
:1058E00025280BD052460D9990476D1C761C2878C0
:1058F0000028F5D10FB03046BDE8F08F0024A04657
:105900000122604900E0044315F8013F203B02FA00
:1059100003F00842F7D128782E2817D115F8010F87
:1059200044F004042A280ED06FF02F022878A0F14A
:10593000300109290AD808EB880102EB410100EB8C
:1059400001086D1CF2E757F8048B6D1C2878692854
:105950003ED006DC0028CDD063280BD0642804D1CB
:1059600036E0732810D075284BD052460D999047D9
:10597000761C85E017F8040B8DF8000000208DF8E8
:105980000100E946012003E057F8049B4FF0FF3087
:1059900061074FF0000401D40AE0641C44450DDAAD
:1059A0008442FADB19F804100029F6D106E0641CE1
:1059B0008442FCDB19F804100029F8D1264404E0E5
:1059C00019F8010B52460D999047641EF8D257E022
:1059D00001CF4FF00A0B002802DA40422D2102E0ED
:1059E000210504D52B218DF82410012103E0E107C6
:1059F00005D02021F7E70DF1200908910CE00021E6
:105A0000F9E701CF4FF00A0BF9E75946FAF747FCDF
:105A100001F1300209F8012D0028F6D1ADEB0900A3
:105A200000F1200B600701D44FF00108D84502DDDA
:105A3000A8EB0B0000E000208046002406E009A847
:105A40005246005D0D999047641C761C089884426C
:105A5000F5DB04E0302052460D999047761CB8F1F2
:105A60000001A8F10108F5DC05E019F8010B524628
:105A70000D999047761CBBF10001ABF1010BF4DCF2
:105A80006D1C34E70928010038B5044601201023B5
:105A90002246122100900520FFF793F838BD000040
:105AA00000B585B02C48007803281DD12BA30FCB5F
:105AB000CDE90323CDE901012748C07804280AD1A4
:105AC0000020102301AA01460090FFF77AF8012078
:105AD0002649087007E00120102301AA0021009048
:105AE0000846FFF76EF835E01B48007804280CD113
:105AF0001FA207CA02AB07C30120102302AA00217C
:105B000000900846FFF75DF824E013480078052868
:105B10000FD11AA0D0E900128068CDE902120490DA
:105B20000120102302AA002100900846FFF749F83F
:105B300010E00948007806280CD113A207CA02AB6E
:105B400007C30120102302AA002100900846FFF796
:105B500038F800BF05B000BD0C0200204D41433AAB
:105B6000313031302E2E2E303030330039010020CC
:105B700048656C6C6F204C322100000048656C6CED
:105B80006F204C332100000048656C6C6F204C3452
:105B9000210000001CB508A00068019007A0006863
:105BA000009002236A46194601A803F06BF91420FD
:105BB000FAF71EFC1CBD000066000000030B00008D
:105BC00070B502460B464FF6FF7000210FE0555CA2
:105BD0006840002508E000F00104401014B14AF2CA
:105BE0000106704080B26D1C082DF4D3491C994207
:105BF000EDD370BD30B585B004460020019003940C
:105C00000120049000200090FBF79CFB694601A84E
:105C1000FBF7DEFA0546FBF733FB05B900BF05B01D
:105C200030BD000007B52548007820B1FEF7EEFC36
:105C30000020224908709DF8000088B920480078AB
:105C400018B12048FFF720FF36E01F48007818B150
:105C5000029800F049F82FE0002000F045F82BE012
:105C60009DF80000012802D102F0E4FC24E09DF838
:105C70000000022802D1FFF703F91DE09DF80000A3
:105C8000032806DB9DF80000062802DCFFF708FF6A
:105C900012E09DF80000072802D103F039F90BE06B
:105CA0009DF80000082807DB9DF800000B2803DCA6
:105CB0009DE8070003F0C0FB0EBD0000F0000020CF
:105CC000F1000020F20000206C01002013B50C460A
:105CD0004FF6FF73012269460248FDF78BFB0098DF
:105CE0001CBD00008817002001B582B001200C23E4
:105CF000FE4A1D2100900E20FEF763FF01200C23B9
:105D0000FB4A1D2100902C20FEF75BFF01200C2395
:105D1000F84A1D2100904A20FEF753FF01200C2372
:105D2000F54A1D2100906820FEF74BFF41F2F0126A
:105D30000298811A904201F0D5847ADC40F6117203
:105D4000A0EB0201904275D038DCB0F5887F72D0AC
:105D500018DCF02870D009DC01286ED00F286DD037
:105D600010286CD0112842F0D483A7E1FF2867D017
:105D7000B0F5807F7DD0A0F2011000287AD00E28E7
:105D8000F1D161E240F2FF12811A904273D00ADC35
:105D9000A0F2111000286FD00E286ED0DF286DD031
:105DA000E028E0D1DBE3A1F60151002967D0012909
:105DB00066D00F2965D01029D5D107E3B1F5877FCB
:105DC0006FD015DCEF296DD008DC0E296BD0DF29F0
:105DD0006AD0E02969D0EE29C5D1C5E3F02972D097
:105DE000FE2971D0FF2970D0B1F5807FBBD1FDE3D2
:105DF000B1F5F87F01F06D820BDCA1F2DF11002913
:105E000077D0012976D00F2975D01029ABD101F0B8
:105E1000A3B9B1F5FF7F01F05D82A1F2FF11002966
:105E200001F05F84012901F063860F299BD101F005
:105E300060BE06E095E3C6E2F9E0A8E0A8E0F5E080
:105E40003DE14DF60F72881A914276D05DDC40F646
:105E50000162A1EB0200914201F0508636DC40F66F
:105E60001F52A1EB0200914201F036821EDC012993
:105E700008E09DE1E6E173E36FE36FE3A5E298E1FB
:105E8000E3E1E0E101F036860F2901F03486B1F557
:105E9000516F01F06381A1F6115100298CD101F0FD
:105EA0001ABAEFE3EFE35DE38EE25CE3012801F071
:105EB0001A84022801F02086102801F01E86E128AD
:105EC0008AD101F011BCFDE3FDE3FDE34DF21F02B9
:105ED000811A90427ED00FDC0E2801F01086A0F5CA
:105EE00050400F38002876D0012875D00F288DD16A
:105EF000EBE3EBE3EBE3EBE301296ED00F296DD08D
:105F0000E0296CD0E12991D1FEE340F60162811ACB
:105F1000904201F022811FDC122801F0F1850DDC96
:105F2000012801F01C81022801F0D781102801F01E
:105F3000D5811128B2D101F0D8BBE6E3202801F0C9
:105F4000E085F12801F0D283F22801F0DB85B0F57D
:105F5000807FA3D101F0D7BD1F2901F0D6850CDCCD
:105F6000012901F0BC810F2901F0BA81102901F04B
:105F7000BE83112992D101F0C7BDF02901F0B88389
:105F8000F12901F0C385FF2988D101F0C0BD00BF10
:105F900001200C23594A082100900846FEF711FE03
:105FA00001200C23554A082100902620FEF709FE07
:105FB00001200C23514A082100904420FEF701FEE5
:105FC0004F48007880B30298012818D14D49142316
:105FD0001A4605E0FEE3FEE3FEE3FEE3FEE3FEE336
:105FE000CDE9001006216420FEF780FD012010237A
:105FF0000B222E2100906620FEF7D0FC14E00298C0
:106000000F2811D10120404914231A46CDE9001070
:1060100006216420FEF76AFD012010230C222E21A8
:1060200000906620FEF7BAFC02F094BA00BF01208F
:106030000C23324A082100900846FEF7C2FD0120D9
:106040000C232E4A082100902620FEF7BAFD0120DD
:106050000C232A4A082100906220FEF7B2FD2B484B
:10606000007850B30298102812D10120254914233A
:106070001A46CDE9001006214620FEF737FD012023
:1060800010230B222E2100904820FEF787FC14E0FD
:106090000298F02811D101201B4914231A46CDE99A
:1060A000001006214620FEF721FD012010230C22BE
:1060B0002E2100904820FEF771FCB5E700BF0120BB
:1060C0000C230E4A082100900846FEF77AFD0120B5
:1060D0000C230A4A082100902620FEF772FD0B4887
:1060E0000078E0B306480078C8B311E02D01002025
:1060F0003001002033010020360100203D01002046
:106100003C010020000000203C0000203B0100205A
:106110000298112824D10120FE4914231A46CDE902
:10612000001006214620FEF7E1FC012010230B227F
:106130002E2100904820FEF731FC0120F549142360
:106140001A46CDE9001006216420FEF7CFFC01209D
:1061500010230B222E2100906620FEF71FFC26E064
:106160000298FF2823D10120EB4914231A46CDE9D8
:10617000001006214620FEF7B9FC012010230C2256
:106180002E2100904820FEF709FC0120E24914234B
:106190001A46CDE9001006216420FEF7A7FC012075
:1061A00010230C222E2100906620FEF7F7FB3BE720
:1061B00000BF01200C23D94A082100900846FEF7B1
:1061C00000FD01200C23D54A082100904420FEF751
:1061D000F8FC01200C23D14A082100906220FEF730
:1061E000F0FCCF48007860B30298B0F5807F12D100
:1061F0000120C84914231A46CDE9001006212820A1
:10620000FEF774FC012010230B222E2100902A207F
:10621000FEF7C4FB15E00298B0F5706F11D10120B4
:10622000BD4914231A46CDE9001006212820FEF7A7
:106230005DFC012010230C222E2100902A20FEF765
:10624000ADFBF1E600BF00BF00BF01200C23B34A45
:10625000082100900846FEF7B4FC01200C23AF4A49
:10626000082100904420FEF7ACFCAD48007858B3FC
:10627000AC48007840B340F201110298884224D122
:106280000120A44914231A46CDE900100621282034
:10629000FEF72CFC012010230B222E2100902A2037
:1062A000FEF77CFB01209B4914231A46CDE9001020
:1062B00006216420FEF71AFC012010230B222E2158
:1062C00000906620FEF76AFB7CE040F60F710298B2
:1062D000884224D10120904914231A46CDE90010A8
:1062E00006212820FEF702FC012010230C222E217B
:1062F00000902A20FEF752FB0120874914231A46FA
:10630000CDE9001006216420FEF7F0FB01201023E8
:106310000C222E2100906620FEF740FB52E040F256
:106320000F110298884224D101207A4914231A4679
:10633000CDE9001006212820FEF7D8FB012010230C
:106340000B222E2100902A20FEF728FB0120724903
:1063500014231A46CDE9001006216420FEF7C6FB7F
:10636000012010230C222E2100906620FEF716FB40
:1063700028E040F601710298884223D10120664945
:1063800014231A46CDE9001006212820FEF7AEFBA3
:10639000012010230C222E2100902A20FEF7FEFA65
:1063A00001205C4914231A46CDE90010062164201F
:1063B000FEF79CFB012010230B222E21009066206B
:1063C000FEF7ECFA30E600BF00BF00BF01200C234F
:1063D000524A082100900846FEF7F3FB01200C23E7
:1063E0004E4A082100906220FEF7EBFB4C480078F3
:1063F00050B34D48007838B30298B0F5887F24D167
:106400000120444914231A46CDE900100621282012
:10641000FEF76CFB012010230B222E2100902A2076
:10642000FEF7BCFA01203B4914231A46CDE90010BF
:1064300006214620FEF75AFB012010230B222E21B5
:1064400000904820FEF7AAFA86E00298B0F57F6F28
:1064500024D10120304914231A46CDE90010062129
:106460002820FEF743FB012010230C222E21009050
:106470002A20FEF793FA0120274914231A46CDE972
:10648000001006214620FEF731FB012010230C22CC
:106490002E2100904820FEF781FA5DE00298B0F5C9
:1064A000F87F24D101201B4914231A46CDE900109E
:1064B00006212820FEF71AFB012010230B222E2193
:1064C00000902A20FEF76AFA0120134914231A4685
:1064D000CDE9001006214620FEF708FB012010231D
:1064E0000C222E2100904820FEF758FA34E0029842
:1064F000B0F5716F30D10120074914231A46CDE958
:10650000001006212820FEF7F1FA012010230C22AA
:106510002E210BE0000000203C0000203D01002067
:106520003A0100203C0100203B01002000902A207D
:10653000FEF734FA0120FE4914231A46CDE9001073
:1065400006214620FEF7D2FA012010230B222E212D
:1065500000904820FEF722FA66E500BF00BF00BFAA
:1065600000BF00BF00BF00BF01200C23F14A08217B
:1065700000900846FEF725FBEF480078002844D03D
:10658000EE4800780028FAD0ED4800780028F6D0D0
:1065900040F211110298884238D10120E4491423B5
:1065A0001A46CDE9001006212820FEF79FFA0120A7
:1065B00010230B222E2100902A20FEF7EFF9012054
:1065C000DB4914231A46CDE9001006214620FEF7C8
:1065D0008DFA012010230B222E2100904820FEF777
:1065E000DDF90120D24914231A4600E0ACE3CDE9DD
:1065F000001006216420FEF779FA012010230B22F7
:106600002E2100906620FEF7C9F9C3E140F21F1168
:106610000298884238D10120C54914231A46CDE991
:10662000001006212820FEF761FA012010230B221A
:106630002E2100902A20FEF7B1F90120BC49142335
:106640001A46CDE9001006214620FEF74FFA012038
:1066500010230B222E2100904820FEF79FF90120E5
:10666000B84914231A46CDE9001006216420FEF72C
:106670003DFA012010230C222E2100906620FEF707
:106680008DF987E161E386E140F2F11102988842D9
:1066900041D10120A64914231A46CDE90010062154
:1066A0002820FEF723FA012010230B222E21009030
:1066B0002A20FEF773F90120A24914231A46CDE9D6
:1066C000001006E0B1E1B2E170E2AFE170E23DE35B
:1066D0003DE306214620FEF709FA012010230C2293
:1066E0002E2100904820FEF759F9012090491423EB
:1066F0001A46CDE9001006216420FEF7F7F90120C3
:1067000010230B222E2101E024E324E300906620D5
:10671000FEF744F93EE140F2FF110298884236D17B
:106720000120834914231A46CDE9001006212820B0
:10673000FEF7DCF9012010230B222E2100902A20E5
:10674000FEF72CF901207F4914231A46CDE90010E9
:1067500006214620FEF7CAF9012010230C222E2123
:1067600000904820FEF71AF90120764914231A46B2
:10677000CDE9001006216420FEF7B8F901201023AE
:106780000C222E2100906620FEF708F902E140F667
:106790001171029888423DD101206A4914231A469A
:1067A000CDE9001006212820FEF7A0F901201023D2
:1067B0000C222E2100902A20FEF7F0F801205C49DF
:1067C00014231A46CDE9001006214620FEF78EF963
:1067D000012005E0EDE1DFE02AE1B9E2B9E2E6E11E
:1067E00010230B222E2100904820FEF7D7F801201D
:1067F0004F4914231A46CDE9001006216420FEF704
:1068000075F9012010230B222E2100906620FEF73F
:10681000C5F8BFE040F61F710298884236D10120CA
:10682000484914231A46CDE9001006212820FEF716
:106830005DF9012010230C222E2100902A20FEF762
:10684000ADF801203A4914231A46CDE9001006217B
:106850004620FEF74BF9012010230B222E21009039
:106860004820FEF79BF80120364914231A46CDE94B
:10687000001006216420FEF739F9012010230C22B4
:106880002E2100906620FEF789F883E040F6F17132
:106890000298884236D101202A4914231A46CDE9AC
:1068A000001006212820FEF721F9012010230C22D8
:1068B0002E2100902A20FEF771F80120214914238F
:1068C0001A46CDE9001006214620FEF70FF90120F7
:1068D00010230C222E2100904820FEF75FF80120A3
:1068E000134914231A46CDE9001006216420FEF74F
:1068F000FDF8012010230B222E2100906620FEF7C8
:106900004DF847E040F6FF710298884242D10120DD
:106910000C4914231A46CDE9001006212820FEF761
:10692000E5F8012010230C222E2100902A200BE0F4
:10693000000000203D0100203A0100203B01002022
:106940003C0100203C000020FEF728F80120F84917
:1069500014231A46CDE9001006214620FEF7C6F89A
:10696000012010230C222E2100904820FEF716F85B
:106970000120EF4914231A46CDE9001006216420B6
:10698000FEF7B4F8012010230C222E21009066207F
:10699000FEF704F80BE400BF01200C23E54A0821B0
:1069A00000902620FEF70DF901200C23E14A082172
:1069B00000904420FEF705F901200C23DD4A082150
:1069C00000906220FEF7FDF8DB48007860B3029883
:1069D000B0F5805F12D10120D84914231A46CDE9C1
:1069E000001006210A20FEF781F8012010230B2257
:1069F0002E2100900C20FDF7D1FF15E00298B0F594
:106A0000704F11D10120CA4914231A46CDE9001054
:106A100006210A20FEF76AF8012010230C222E21FD
:106A200000901046FDF7BAFF0BE400BF00BF00BFA7
:106A300001200C23BF4A082100902620FEF7C1F850
:106A400001200C23BB4A082100904420FEF7B9F82E
:106A5000B948007858B3BA48007840B341F2010110
:106A60000298884224D10120B44914231A46CDE962
:106A7000001006210A20FEF739F8012010230B220E
:106A80002E2100900C20FDF789FF0120AB49142333
:106A90001A46CDE9001006216420FEF727F80120F0
:106AA00010230B222E2100906620FDF777FF7CE05B
:106AB0004FF20F010298884224D101209C491423EF
:106AC0001A46CDE9001006210A20FEF70FF8012032
:106AD00010230C222E2100901046FDF75FFF0120AD
:106AE000934914231A46CDE9001006216420FDF7CE
:106AF000FDFF012010230C222E2100906620FDF7BF
:106B00004DFF52E041F20F010298884224D101204A
:106B10008A4914231A46CDE9001006210A20FDF700
:106B2000E5FF012010230B222E2100900C20FDF701
:106B300035FF01207E4914231A46CDE900100621B5
:106B40006420FDF7D3FF012010230C222E2100909A
:106B50006620FDF723FF28E04FF2010102988842EA
:106B600023D10120724914231A46CDE900100621D1
:106B70000A20FDF7BBFF012010230C222E210090DC
:106B80001046FDF70BFF01206C4914231A46CDE98E
:106B9000001006216420FDF7A9FF012010230B221D
:106BA0002E2100906620FDF7F9FE0BE400BF00BF28
:106BB00000BF01200C235F4A082100902620FEF729
:106BC00000F801200C235B4A082100906220FDF7A9
:106BD000F8FF5948007858B35A48007840B341F25A
:106BE00010010298884224D10120544914231A46E6
:106BF000CDE9001006210A20FDF778FF01201023BF
:106C00000B222E2100900C20FDF7C8FE01204B49DD
:106C100014231A46CDE9001006214620FDF766FF31
:106C2000012010230B222E2100904820FDF7B6FEF4
:106C30007CE04FF2F0010298884224D101203C49C7
:106C400014231A46CDE9001006210A20FDF74EFF55
:106C5000012010230C222E2100901046FDF79EFEED
:106C60000120334914231A46CDE90010062146209D
:106C7000FDF73CFF012010230C222E21009048201C
:106C8000FDF78CFE52E041F2F0010298884224D1D7
:106C900001202A4914231A46CDE9001006210A20B2
:106CA000FDF724FF012010230B222E2100900C2041
:106CB000FDF774FE01201E4914231A46CDE9001089
:106CC00006214620FDF712FF012010230C222E2161
:106CD00000904820FDF762FE28E04FF21001029874
:106CE000884223D10120124914231A46CDE900100D
:106CF00006210A20FDF7FAFE012010230C222E2186
:106D000000901046FDF74AFE01200C4914231A4654
:106D1000CDE9001006214620FDF7E8FE01201023F2
:106D20000B222E2100904820FDF738FE14E40000CD
:106D30003C0000203D01002039010020000000201F
:106D40003C0100203B01002000BF00BF00BF00BF8E
:106D500000BF00BF00BF01200C23F94A08210090AA
:106D60002620FDF72EFFF7480078002842D0F6488D
:106D700000780028FAD0F54800780028F6D041F2D3
:106D800011010298884236D10120F14914231A4694
:106D9000CDE9001006210A20FDF7A8FE01201023EE
:106DA0000B222E2100900C20FDF7F8FD0120E84970
:106DB00014231A46CDE9001006214620FDF796FE61
:106DC000012010230B222E2100904820FDF7E6FD24
:106DD0000120DF4914231A46CDE900100621642062
:106DE000FDF784FE012010230B222E210090662047
:106DF000FDF7D4FDA2E141F21F010298884236D18D
:106E00000120D34914231A46CDE9001006210A2097
:106E1000FDF76CFE012010230B222E2100900C2088
:106E2000FDF7BCFD0120CA4914231A46CDE9001024
:106E300006214620FDF75AFE012010230B222E21A9
:106E400000904820FDF7AAFD0120C24914231A46EC
:106E5000CDE9001006216420FDF748FE0120102333
:106E60000C222E2100906620FDF798FD66E141F28C
:106E7000F1010298884236D10120B54914231A46FF
:106E8000CDE9001006210A20FDF730FE0120102375
:106E90000B222E2100900C20FDF780FD0120AD4932
:106EA00014231A46CDE9001006214620FDF71EFEE8
:106EB000012010230C222E2100904820FDF76EFDAA
:106EC0000120A34914231A46CDE9001006216420AD
:106ED000FDF70CFE012010230B222E2100906620CE
:106EE000FDF75CFD2AE141F2FF010298884236D1AC
:106EF0000120974914231A46CDE9001006210A20E3
:106F0000FDF7F4FD012010230B222E2100900C2010
:106F1000FDF744FD01208F4914231A46CDE90010E6
:106F200006214620FDF7E2FD012010230C222E2130
:106F300000904820FDF732FD0120864914231A46AF
:106F4000CDE9001006216420FDF7D0FD01201023BB
:106F50000C222E2100906620FDF720FDEEE04FF27E
:106F600011010298884236D101207A4914231A4629
:106F7000CDE9001006210A20FDF7B8FD01201023FD
:106F80000C222E2100901046FDF708FD01207049CB
:106F900014231A46CDE9001006214620FDF7A6FD70
:106FA000012010230B222E2100904820FDF7F6FC33
:106FB0000120674914231A46CDE9001006216420F8
:106FC000FDF794FD012010230B222E210090662056
:106FD000FDF7E4FCB2E04FF21F010298884236D17F
:106FE00001205C4914231A46CDE9001006210A202D
:106FF000FDF77CFD012010230C222E21009010466D
:10700000FDF7CCFC0120524914231A46CDE90010AB
:1070100006214620FDF76AFD012010230B222E21B8
:1070200000904820FDF7BAFC01204A4914231A4673
:10703000CDE9001006216420FDF758FD0120102342
:107040000C222E2100906620FDF7A8FC76E04FF27E
:10705000F1010298884236D101203E4914231A4694
:10706000CDE9001006210A20FDF740FD0120102384
:107070000C222E2100901046FDF790FC012035498E
:1070800014231A46CDE9001006214620FDF72EFDF7
:10709000012010230C222E2100904820FDF77EFCB9
:1070A00001202B4914231A46CDE900100621642043
:1070B000FDF71CFD012010230B222E2100906620DD
:1070C000FDF76CFC3AE04FF2FF010298884235D19F
:1070D0000120204914231A46CDE9001006210A2078
:1070E000FDF704FD012010230C222E2100901046F4
:1070F000FDF754FC0120174914231A46CDE900106E
:1071000006214620FDF7F2FC012010230C222E213F
:1071100000904820FDF742FC01200E4914231A4636
:10712000CDE9001006216420FDF7E0FC01201023CA
:107130000C222E2100906620FDF730FC2AE400008E
:107140003D010020390100203B0100203C010020CE
:10715000000000203C00002000BF00BF00BF012055
:107160000C23FE4A082100904420FDF72AFD01204F
:107170000C23FA4A082100906220FDF722FDF8480E
:10718000007850B3F748007838B30298B0F5885FBC
:1071900024D10120F44914231A46CDE90010062118
:1071A0000A20FDF7A3FC012010230B222E210090C2
:1071B0000C20FDF7F3FB0120EB4914231A46CDE91F
:1071C000001006212820FDF791FC012010230B223E
:1071D0002E2100902A20FDF7E1FB79E00298B0F51E
:1071E0007F4F24D10120E14914231A46CDE9001034
:1071F00006210A20FDF77AFC012010230C222E2103
:1072000000901046FDF7CAFB0120D84914231A4606
:10721000CDE9001006212820FDF768FC012010238D
:107220000C222E2100902A20FDF7B8FB50E0029896
:10723000B0F5F85F24D10120CB4914231A46CDE9DB
:10724000001006210A20FDF751FC012010230B221B
:107250002E2100900C20FDF7A1FB0120C34914232F
:107260001A46CDE9001006212820FDF73FFC012039
:1072700010230C222E2100902A20FDF78FFB27E0FF
:107280000298B0F5714F23D10120B84914231A4652
:10729000CDE9001006210A20FDF728FC012010236B
:1072A0000C222E2100901046FDF778FB0120AE49FC
:1072B00014231A46CDE9001006212820FDF716FCFC
:1072C000012010230B222E2100902A20FDF766FBBF
:1072D0006BE400BF00BF00BF00BF00BF00BF00BF26
:1072E00001200C239D4A082100904420FDF769FCF1
:1072F0009B480078002842D09A4800780028FAD0AD
:107300009B4800780028F6D041F20111029888428B
:1073100036D10120944914231A46CDE900100621E4
:107320000A20FDF7E3FB012010230B222E21009001
:107330000C20FDF733FB01208B4914231A46CDE9BD
:10734000001006212820FDF7D1FB012010230B227D
:107350002E2100902A20FDF721FB012082491423D1
:107360001A46CDE9001006216420FDF7BFFB01207D
:1073700010230B222E2100906620FDF70FFBAFE1BA
:1073800041F20F110298884236D101207649142328
:107390001A46CDE9001006210A20FDF7A7FB0120BF
:1073A00010230B222E2100900C20FDF7F7FA01206C
:1073B0006D4914231A46CDE9001006212820FDF757
:1073C00095FB012010230B222E2100902A20FDF78F
:1073D000E5FA0120654914231A46CDE9001006217B
:1073E0006420FDF783FB012010230C222E21009046
:1073F0006620FDF7D3FA73E141F6017102988842E5
:1074000036D10120584914231A46CDE9001006212F
:107410000A20FDF76BFB012010230B222E21009088
:107420000C20FDF7BBFA0120504914231A46CDE980
:10743000001006212820FDF759FB012010230C2203
:107440002E2100902A20FDF7A9FA01204649142395
:107450001A46CDE9001006216420FDF747FB012004
:1074600010230B222E2100906620FDF797FA37E1BA
:1074700041F60F710298884236D101203A4914230F
:107480001A46CDE9001006210A20FDF72FFB012046
:1074900010230B222E2100900C20FDF77FFA0120F3
:1074A000324914231A46CDE9001006212820FDF7A1
:1074B0001DFB012010230C222E2100902A20FDF715
:1074C0006DFA0120294914231A46CDE9001006213E
:1074D0006420FDF70BFB012010230C222E210090CD
:1074E0006620FDF75BFAFBE04FF20111029888423B
:1074F00043D101201D4914231A46CDE9001006216D
:107500000A20FDF7F3FA012010230C222E2100900F
:107510001046FDF743FA0120134914231A46CDE91A
:10752000001006212820FDF7E1FA012010230B228C
:107530002E2100902A20FDF731FA01200A49142358
:107540001A46CDE9001006216420FDF7CFFA01208C
:1075500010230B222E21009066200BE03D0100201D
:10756000390100203A010020000000203C000020EA
:107570003C010020FDF712FAB2E04FF20F11029821
:10758000884236D10120FA4914231A46CDE9001069
:1075900006210A20FDF7AAFA012010230C222E2131
:1075A00000901046FDF7FAF90120F24914231A461B
:1075B000CDE9001006212820FDF798FA01201023BC
:1075C0000B222E2100902A20FDF7E8F90120E8493E
:1075D00014231A46CDE9001006216420FDF786FA2F
:1075E000012010230C222E2100906620FDF7D6F9F1
:1075F00076E04FF601710298884236D10120DC49CD
:1076000014231A46CDE9001006210A20FDF76EFA70
:10761000012010230C222E2100901046FDF7BEF908
:107620000120D34914231A46CDE900100621282051
:10763000FDF75CFA012010230C222E2100902A2055
:10764000FDF7ACF90120CB4914231A46CDE900100F
:1076500006216420FDF74AFA012010230B222E2177
:1076600000906620FDF79AF93AE04FF60F71029804
:10767000884235D10120BE4914231A46CDE90010B5
:1076800006210A20FDF732FA012010230C222E21B8
:1076900000901046FDF782F90120B54914231A46DF
:1076A000CDE9001006212820FDF720FA0120102343
:1076B0000C222E2100902A20FDF770F90120AC4900
:1076C00014231A46CDE9001006216420FDF70EFAB6
:1076D000012010230C222E2100906620FDF75EF978
:1076E0002CE500BF00BF00BF00BF00BF00BF00BF50
:1076F00001200C23A04A082100906220FDF761FAC6
:107700009E480078002842D09D4800780028FAD092
:107710009C4800780028F6D041F210110298884267
:1077200036D10120934914231A46CDE900100621D1
:107730000A20FDF7DBF9012010230B222E210090F7
:107740000C20FDF72BF901208A4914231A46CDE9B4
:10775000001006214620FDF7C9F9012010230B2255
:107760002E2100904820FDF719F9012081491423AA
:107770001A46CDE9001006212820FDF7B7F90120AF
:1077800010230B222E2100902A20FDF707F9AEE1ED
:1077900041F2F0110298884236D101207549142334
:1077A0001A46CDE9001006210A20FDF79FF90120B5
:1077B00010230B222E2100900C20FDF7EFF8012062
:1077C0006C4914231A46CDE9001006212820FDF744
:1077D0008DF9012010230B222E2100902A20FDF785
:1077E000DDF80120624914231A46CDE90010062174
:1077F0004620FDF77BF9012010230C222E2100905A
:107800004820FDF7CBF872E141F6107102988842EA
:1078100036D10120574914231A46CDE9001006211C
:107820000A20FDF763F9012010230B222E2100907E
:107830000C20FDF7B3F801204D4914231A46CDE979
:10784000001006212820FDF751F9012010230C22F9
:107850002E2100902A20FDF7A1F80120454914238C
:107860001A46CDE9001006214620FDF73FF9012018
:1078700010230B222E2100904820FDF78FF836E1CF
:1078800041F6F0710298884236D10120394914231B
:107890001A46CDE9001006210A20FDF727F901203C
:1078A00010230B222E2100900C20FDF777F80120E9
:1078B0002F4914231A46CDE9001006212820FDF790
:1078C00015F9012010230C222E2100902A20FDF70B
:1078D00065F80120264914231A46CDE90010062137
:1078E0004620FDF703F9012010230C222E210090E1
:1078F0004820FDF753F8FAE04FF210110298884241
:1079000042D101201A4914231A46CDE9001006215C
:107910000A20FDF7EBF8012010230C222E21009005
:107920001046FDF73BF80120124914231A46CDE911
:10793000001006212820FDF7D9F8012010230B2282
:107940002E2100902A20FDF729F80120094914234F
:107950001A46CDE9001006214620FDF7C7F80120A0
:1079600010230B222E2100904820FDF717F8BEE0CF
:107970003C000020000000203D01002039010020D3
:107980003A0100203C0100204FF2F0110298884299
:1079900036D10120FE4914231A46CDE900100621F4
:1079A0000A20FDF7A3F8012010230C222E210090BD
:1079B0001046FCF7F3FF0120F64914231A46CDE9DF
:1079C000001006212820FDF791F8012010230B223A
:1079D0002E2100902A20FCF7E1FF0120EC4914231E
:1079E0001A46CDE9001006214620FDF77FF8012058
:1079F00010230C222E2100904820FCF7CFFF76E0C8
:107A00004FF610710298884236D10120E0491423C4
:107A10001A46CDE9001006210A20FDF767F801207B
:107A200010230C222E2100901046FCF7B7FF0120F6
:107A3000D74914231A46CDE9001006212820FDF766
:107A400055F8012010230C222E2100902A20FCF74B
:107A5000A5FF0120CF4914231A46CDE900100621C5
:107A60004620FDF743F8012010230B222E21009021
:107A70004820FCF793FF3AE04FF6F07102988842F5
:107A800035D10120C24914231A46CDE90010062140
:107A90000A20FDF72BF8012010230C222E21009044
:107AA0001046FCF77BFF0120B94914231A46CDE9A3
:107AB000001006212820FDF719F8012010230C22C0
:107AC0002E2100902A20FCF769FF0120B0491423E1
:107AD0001A46CDE9001006214620FDF707F80120DF
:107AE00010230C222E2100904820FCF757FFF7E5C9
:107AF00000BF00BF00BF00BF00BF00BF00BF00BF8E
:107B000000BF00BF00BF00BF00BF00BF00BFA24852
:107B10000078002858D0A14800780028FAD0A04862
:107B200000780028F6D09F4800780028F2D041F273
:107B300011110298884248D10120964914231A460F
:107B4000CDE9001006210A20FCF7D0FF0120102308
:107B50000B222E2100900C20FCF720FF01208D49E4
:107B600014231A46CDE9001006212820FCF7BEFF99
:107B7000012010230B222E2100902A20FCF70EFF5B
:107B80000120844914231A46CDE90010062146201D
:107B9000FCF7ACFF012010230B222E21009048207F
:107BA000FCF7FCFE01207B4914231A46CDE90010A6
:107BB00006216420FCF79AFF012010230B222E21BE
:107BC00000906620FCF7EAFE2DE241F21F110298B8
:107BD000884248D101206F4914231A46CDE900108C
:107BE00006210A20FCF782FF012010230B222E2100
:107BF00000900C20FCF7D2FE0120664914231A469F
:107C0000CDE9001006212820FCF770FF0120102389
:107C10000B222E2100902A20FCF7C0FE01205D4996
:107C200014231A46CDE9001006214620FCF75EFF1A
:107C3000012010230B222E2100904820FCF7AEFEDD
:107C40000120534914231A46CDE90010062164206F
:107C5000FCF74CFF012010230C222E2100906620FF
:107C6000FCF79CFEDFE141F2F1110298884248D115
:107C70000120484914231A46CDE9001006210A20A4
:107C8000FCF734FF012010230B222E2100900C2042
:107C9000FCF784FE01203F4914231A46CDE9001069
:107CA00006212820FCF722FF012010230B222E2181
:107CB00000902A20FCF772FE0120354914231A4651
:107CC000CDE9001006214620FCF710FF012010230B
:107CD0000C222E2100904820FCF760FE01202D4947
:107CE00014231A46CDE9001006216420FCF7FEFE9D
:107CF000012010230B222E2100906620FCF74EFE5F
:107D000091E141F2FF110298884255D101202149A9
:107D100014231A46CDE9001006210A20FCF7E6FEDE
:107D2000012010230B222E2100900C20FCF736FEA0
:107D30000120184914231A46CDE9001006212820F5
:107D4000FCF7D4FE012010230B222E2100902A20C4
:107D5000FCF724FE01200E4914231A46CDE9001039
:107D600006214620FCF7C2FE012010230C222E2102
:107D700000904820FCF712FE0120054914231A4602
:107D8000CDE9001006216420FCF7B0FE01200BE0D5
:107D90003C00002000000020390100203A010020B2
:107DA0003B0100203C01002010230C222E210090DA
:107DB0006620FCF7F3FDABE341F6117102988842AF
:107DC00048D10120FE4914231A46CDE900100621AE
:107DD0000A20FCF78BFE012010230B222E2100909D
:107DE0000C20FCF7DBFD0120F64914231A46CDE9EF
:107DF000001006212820FCF779FE012010230C2218
:107E00002E2100902A20FCF7C9FD0120EC49142303
:107E10001A46CDE9001006214620FCF767FE012036
:107E200010230B222E2100904820FCF7B7FD0120E3
:107E3000E34914231A46CDE9001006216420FCF71B
:107E400055FE012010230B222E2100906620FCF706
:107E5000A5FD5DE341F61F710298884248D10120DB
:107E6000D74914231A46CDE9001006210A20FCF751
:107E70003DFE012010230B222E2100900C20FCF748
:107E80008DFD0120CF4914231A46CDE900100621AB
:107E90002820FCF72BFE012010230C222E2100901D
:107EA0002A20FCF77BFD0120C54914231A46CDE9A1
:107EB000001006214620FCF719FE012010230B229A
:107EC0002E2100904820FCF769FD0120BD491423B4
:107ED0001A46CDE9001006216420FCF707FE0120B8
:107EE00010230C222E2100906620FCF757FD0FE393
:107EF00041F6F1710298884248D10120B04914231B
:107F00001A46CDE9001006210A20FCF7EFFD0120FA
:107F100010230B222E2100900C20FCF73FFD0120A6
:107F2000A84914231A46CDE9001006212820FCF7A1
:107F3000DDFD012010230C222E2100902A20FCF7C9
:107F40002DFD01209F4914231A46CDE9001006217A
:107F50004620FCF7CBFD012010230C222E2100909F
:107F60004820FCF71BFD0120954914231A46CDE952
:107F7000001006216420FCF7B9FD012010230B221C
:107F80002E2100906620FCF709FDC1E241F6FF7149
:107F90000298884248D10120894914231A46CDE924
:107FA000001006210A20FCF7A1FD012010230B225E
:107FB0002E2100900C20FCF7F1FC012081491423B4
:107FC0001A46CDE9001006212820FCF78FFD01207C
:107FD00010230C222E2100902A20FCF7DFFC012028
:107FE000784914231A46CDE9001006214620FCF7F3
:107FF0007DFD012010230C222E2100904820FCF74B
:10800000CDFC01206F4914231A46CDE9001006214A
:108010006420FCF76BFD012010230C222E21009020
:108020006620FCF7BBFC73E24FF211110298884204
:1080300048D10120634914231A46CDE900100621D6
:108040000A20FCF753FD012010230C222E21009062
:108050001046FCF7A3FC0120594914231A46CDE928
:10806000001006212820FCF741FD012010230B22DF
:108070002E2100902A20FCF791FC01205049142366
:108080001A46CDE9001006214620FCF72FFD0120FD
:1080900010230B222E2100904820FCF77FFC0120AA
:1080A000474914231A46CDE9001006216420FCF745
:1080B0001DFD012010230B222E2100906620FCF7CD
:1080C0006DFC25E24FF21F110298884248D1012031
:1080D0003C4914231A46CDE9001006210A20FCF77A
:1080E00005FD012010230C222E2100901046FCF7E4
:1080F00055FC0120324914231A46CDE9001006210F
:108100002820FCF7F3FC012010230B222E210090E5
:108110002A20FCF743FC0120294914231A46CDE903
:10812000001006214620FCF7E1FC012010230B2261
:108130002E2100904820FCF731FC01202149142316
:108140001A46CDE9001006216420FCF7CFFC01207F
:1081500010230C222E2100906620FCF71FFCD7E193
:108160004FF2F111029888424DD101201549142394
:108170001A46CDE9001006210A20FCF7B7FC0120C1
:1081800010230C222E2100901046FCF707FC012042
:108190000B4914231A46CDE9001006212820FCF7CC
:1081A000A5FC012010230B222E2100902A20FCF791
:1081B000F5FB0120034914231A46CDE9001003E022
:1081C000000000203C00002006214620FCF78EFC29
:1081D000012010230C222E2100904820FCF7DEFB0A
:1081E0000120DD4914231A46CDE900100621642040
:1081F000FCF77CFC012010230B222E21009066202E
:10820000FCF7CCFB84E14FF2FF110298884248D181
:108210000120D24914231A46CDE9001006210A2074
:10822000FCF764FC012010230C222E210090104644
:10823000FCF7B4FB0120C84914231A46CDE900100D
:1082400006212820FCF752FC012010230B222E21AE
:1082500000902A20FCF7A2FB0120C04914231A46F3
:10826000CDE9001006214620FCF740FC0120102338
:108270000C222E2100904820FCF790FB0120B749EA
:1082800014231A46CDE9001006216420FCF72EFCC9
:10829000012010230C222E2100906620FCF77EFB8B
:1082A00036E14FF611710298884248D10120AB495E
:1082B00014231A46CDE9001006210A20FCF716FC0B
:1082C000012010230C222E2100901046FCF766FBA3
:1082D0000120A24914231A46CDE9001006212820C6
:1082E000FCF704FC012010230C222E2100902A20F0
:1082F000FCF754FB0120984914231A46CDE90010DD
:1083000006214620FCF7F2FB012010230B222E2130
:1083100000904820FCF742FB01208F4914231A46A5
:10832000CDE9001006216420FCF7E0FB01201023BA
:108330000B222E2100906620FCF730FBE8E04FF680
:108340001F710298884248D10120844914231A469B
:10835000CDE9001006210A20FCF7C8FB01201023FC
:108360000C222E2100901046FCF718FB01207B49BF
:1083700014231A46CDE9001006212820FCF7B6FB8D
:10838000012010230C222E2100902A20FCF706FB4E
:108390000120714914231A46CDE900100621462018
:1083A000FCF7A4FB012010230B222E210090482073
:1083B000FCF7F4FA0120694914231A46CDE90010AC
:1083C00006216420FCF792FB012010230C222E21B1
:1083D00000906620FCF7E2FA9AE04FF6F1710298FD
:1083E000884248D101205D4914231A46CDE9001086
:1083F00006210A20FCF77AFB012010230C222E21F3
:1084000000901046FCF7CAFA0120544914231A467A
:10841000CDE9001006212820FCF768FB012010237D
:108420000C222E2100902A20FCF7B8FA01204B499B
:1084300014231A46CDE9001006214620FCF756FB0E
:10844000012010230C222E2100904820FCF7A6FAD0
:108450000120414914231A46CDE900100621642069
:10846000FCF744FB012010230B222E2100906620F4
:10847000FCF794FA4CE04FF6FF710298884247D11E
:108480000120364914231A46CDE9001006210A209E
:10849000FCF72CFB012010230C222E21009010460B
:1084A000FCF77CFA01202D4914231A46CDE900106F
:1084B00006212820FCF71AFB012010230C222E2174
:1084C00000902A20FCF76AFA0120244914231A4656
:1084D000CDE9001006214620FCF708FB01201023FF
:1084E0000C222E2100904820FCF758FA01201B494D
:1084F00014231A46CDE9001006216420FCF7F6FA91
:10850000012010230C222E2100906620FCF746FA51
:1085100020E001200C23124A082100900846FCF7B5
:1085200050FB01200C230E4A082100902620FCF766
:1085300048FB01200C230A4A082100904420FCF744
:1085400040FB01200C23064A082100906220FCF722
:1085500038FB00BF00BF0EBD000000203C00002023
:108560003D0100201CB508A00068019007A000682C
:10857000009002236A46194601A800F083FC1420EB
:10858000F7F736FF1CBD0000660000000100000088
:10859000F9F7BAF8FCF720FEFBF7B0FDFBF710FD8A
:1085A000FBF7F0FEFBF734FFFBF768FFFBF7D6FFA6
:1085B000FBF7F0FFFCF70AF8FBF798FFFBF7B2FFB9
:1085C000FBF704FFFBF7C2FCFBF724FE1148FAF7A8
:1085D000C1F91148FAF7BEF900BFFCF78FF8002087
:1085E000FCF72CF80020FCF737F800BF0B480068B8
:1085F000C06840F0200009490968C86008A10BA0C4
:10860000FDF72AF9FBF724FAFBF73AFD00F0D8F85A
:1086100000BFFEE7E815002030160020BC16002041
:1086200044747553746172742E2E2E0025730D0AD6
:108630000000000008B50120102314220D21009035
:108640000A20FCF7ABF90120102315220D21009020
:108650001B20FCF7A3F901201023274A0D210090CD
:108660002C20FCF7AEFA012010231C220D210090D3
:108670003F20FCF793F9012010231D220D210090CB
:108680005020FCF78BF9012010230D2228210090A7
:108690000A20FCF783F9012010230E2228210090E4
:1086A0002120FCF77BF9012010230F2228210090C4
:1086B0003720FCF773F9012010231A462821009077
:1086C0005020FCF76BF90D484078012808D10020B4
:1086D00010230B4A0D2100906420FCF772FA0AE087
:1086E0000648407838B900201023054A2821009018
:1086F0006420FCF766FA08BD040100200C0200208B
:108700000001002001460020842901D0CA1C104429
:10871000704700007FB586B01EA0006805901EA3BC
:108720000FCB01AC0FC4069C200E8DF80600200C68
:108730008DF80700200A8DF80800E0B28DF80900D6
:10874000079D280E8DF80A00280C8DF80B00280ACA
:108750008DF80C00E8B28DF80D00089E300E8DF8F3
:108760000E00300C8DF80F00300A8DF81000F0B2BA
:108770008DF811009DF824008DF812000F2301AA36
:10878000022105A800F07EFB1420F7F731FE0AB0A5
:1087900070BD000066000000020C00000000000038
:1087A000000000000000000070B5044625460DB131
:1087B000294600E00121084600F06AFD002070BD56
:1087C00010B500F093FD002010BD7FB504460D46A6
:1087D000606998B1A06988B1B4F90800FFF792FF09
:1087E0000646D4E90510CDE9006102902B462269C6
:1087F000D4E9001000F078FF039013E0B4F908000A
:10880000FFF780FF064603A8CDE90060238A9AB2ED
:108810002B46D4E9001000F035FF012802D00020DB
:1088200004B070BD0398FBE72DE9F04105460E4604
:108830001C4807681C480068001D00F02DFC50B95A
:108840001948006890F82C100120884017490968E1
:10885000814316480160681C38B936B11248016876
:10886000091D134800F062FC1AE07C190E480068EC
:108870004460BC4207D20C480168091D0D480068DD
:1088800000F03AFC0CE008480168091D0A4800683D
:1088900000F032FC09480068844201D207480460B5
:1088A000BDE8F081BC010020A8010020C00100202B
:1088B000341B0020B0010020AC010020D8010020B2
:1088C00010B5044600F03EFC23480068401C2249D5
:1088D00008602248006840B92048046008460068E3
:1088E00001280DD100F03AF90AE01D48006838B9B6
:1088F0001A480068C06AE16A884201D817480460D3
:1089000018480068401C1749086094F82C10012092
:10891000884015490968084313490860E16A01EB7A
:108920008101124A02EB8100211D00F0FFFB00F0E3
:1089300033FC0B48006868B108480068C06AE16A07
:10894000884207D24FF0805009490860BFF34F8F2B
:10895000BFF36F8F10BD0000B8010020A8010020F8
:10896000C4010020D4010020C0010020581A0020BA
:1089700004ED00E010B516E000F0E4FB0C48C06820
:10898000C468201D00F088FB0A480068401E0949A1
:10899000086009480068401E0749086000F0FCFBB9
:1089A000204600F00BF8044800680028E4D110BD10
:1089B000201B0020B8010020B401002010B504469F
:1089C00094F8510030B9206B00F004FC204600F010
:1089D00001FC1AE094F85100012803D1204600F070
:1089E000F9FB12E094F85100022801D1012000E0C7
:1089F000002050B900BF502080F31188BFF34F8F83
:108A0000BFF36F8F00BF00BFFEE710BD30B54FF45E
:108A10004063174800F007042CB1C01D20F0070088
:108A2000134C041B1B1B0246124C22600024114DE8
:108A30006C60D018083820F007000F4C206000242C
:108A40000D4D2D686C600C4D2D682C601146441A3C
:108A50004C60094C24680C60084D4C682C60084D33
:108A60004C682C604FF00044064D2C6030BD000077
:108A7000481B0020E4010020EC010020F40100204C
:108A8000F0010020F801002000BFFFF773FF064847
:108A900000680128F9D94FF0805004490860BFF3FD
:108AA0004F8FBFF36F8FF0E7581A002004ED00E0FE
:108AB0002DE9FF5F81460F469246DDE90E6B109C63
:108AC000AAF10100216B01EB800828F0070808F0EB
:108AD000070008B9012000E0002050B900BF502075
:108AE00080F31188BFF34F8FBFF36F8F00BF00BFBC
:108AF000FEE7002507E0795D04F134004155785D1B
:108B000000B902E06D1C102DF5D300BF00214320F9
:108B10000155072E00D30626E66266640020A06495
:108B2000201D00F0E6FA04F1180000F0E2FA2461DA
:108B3000C6F10700A06164620020E06484F8500080
:108B400049464046039A00F049F92060BBF1000F06
:108B500001D0CBF80040BDE8FF9F000010B5002415
:108B600007E004EB84010F4A02EB810000F0B4FA45
:108B7000641C072CF5D30C4800F0AEFA0B4800F04B
:108B8000ABFA0B4800F0A8FA0A4800F0A5FA0A4828
:108B900000F0A2FA0448094908600448084908603E
:108BA00010BD0000581A0020E41A0020F81A002016
:108BB0000C1B0020201B0020341B0020AC010020D7
:108BC000B001002010B50146164800E000680368B7
:108BD0008B42FBD30246436813448B4204D1436863
:108BE0004C682344436001460A464B6813440468BA
:108BF000A34211D10C4C03682468A34208D04B68EF
:108C00000468646823444B6003681B680B6005E0DC
:108C1000054B1B680B6001E003680B60884200D0C5
:108C2000016010BDE4010020EC0100200A49096840
:108C3000096809B9012100E0002121B14FF0FF319D
:108C4000064A116006E004490968C968C868034A11
:108C50004168116070470000AC010020D80100207D
:108C60000E480068401C08B9012000E0002050B9FF
:108C700000BF502080F31188BFF34F8FBFF36F8F79
:108C800000BF00BFFEE700BF502080F31188BFF394
:108C90004F8FBFF36F8F00BF00BFFEE7FC010020C6
:108CA0002DE9F04104464FF0000800F077FB4648FC
:108CB000006808B9FFF7AAFE444800682040002871
:108CC0006BD1D4B1083404F00700B0B104F0070050
:108CD000C0F10800044404F0070008B9012000E0D6
:108CE000002050B900BF502080F31188BFF34F8F90
:108CF000BFF36F8F00BF00BFFEE7002C4DD034489C
:108D00000068844249D8334E3046056801E02E465B
:108D10002D686868A04202D228680028F7D12A4846
:108D20000068854239D0306800F108082868306052
:108D30006868001B102819D92F1907F0070008B917
:108D4000012000E0002050B900BF502080F31188BE
:108D5000BFF34F8FBFF36F8F00BF00BFFEE76868A0
:108D6000001B78606C603846FFF72CFF1849686874
:108D70000968081A16490860084600681649096813
:108D8000884203D212480068134908600F49686896
:108D90000968084368600020286000F0A5FD08F01D
:108DA000070008B9012000E0002050B900BF5020A2
:108DB00080F31188BFF34F8FBFF36F8F00BF00BFE9
:108DC000FEE74046BDE8F081EC010020F8010020FC
:108DD000F0010020E4010020F4010020001F4FF00A
:108DE00080730360001F21F001030360001F034B29
:108DF000036014380260203870470000618C00085E
:108E000001460888704700002DE9F047044689466E
:108E100015461E46002700BF21E005EB85004FEAFE
:108E2000400821461048FCF7CFFC1E20F8F7BCF99B
:108E30000E490FA0FCF710FD0AE049460B48F7F772
:108E400015FA10B10120BDE8F0876420F8F7ACF9FD
:108E5000B8F10000A8F10108EFD1781CC7B2B74201
:108E6000DBDB0020EFE70000BC160020A80A002092
:108E70002D2D2D2D2D2D2D2D2D2D2D2D2D2D3E2519
:108E8000730000002DE9F04389B005468846164678
:108E90001C46142104A8F7F7DEF928788DF8100095
:108EA00068788DF811002146304600F09FFD81461C
:108EB0000020009001900290039000BF03E0315C1D
:108EC0000DF80010401CA042F9D30DF804900020CA
:108ED00006E01DF8001000EB080204AB9954401C9A
:108EE0001028F6DB122104A8FCF76AFE0746F8B248
:108EF0008DF82200380A8DF82300142204A90348B3
:108F0000FCF74CFC09B0BDE8F0830000BC16002063
:108F100008B501201023504A022100901420FBF7CD
:108F200050FE01200E231422022100903220FBF774
:108F300035FD01200E231522022100904620FBF76B
:108F40002DFD01201023454A112100901420FBF72C
:108F500038FE01200E231422112100903220FBF74D
:108F60001DFD01200E231522112100904620FBF744
:108F700015FD012010233A4A202100901420FBF710
:108F800020FE01200E231422202100903220FBF726
:108F900005FD01200E231522202100904620FBF71D
:108FA000FDFC012010232F4A2F2100901420FBF7F5
:108FB00008FE01200E2314222F2100903220FBF7FF
:108FC000EDFC01200E2315222F2100904620FBF7F7
:108FD000E5FC2548407804280BD12348807840B927
:108FE00000201023214A022100906420FBF7E9FDB4
:108FF00031E01D48407803280CD11B4880780128B7
:1090000008D100201023194A112100906420FBF799
:10901000D8FD20E01448407802280CD1124880780E
:10902000022808D100201023104A2021009064203B
:10903000FBF7C7FD0FE00C48407801280BD10A4828
:109040008078032807D100201023084A2F210090A0
:109050006420FBF7B6FD08BD070100200B010020CE
:109060000F010020130100200C020020000100204D
:1090700010B5FAF72BFA07490870FAF7B1FA054963
:109080004870FAF737FB03498870FAF735FC014955
:10909000C87010BD4801002001460A69D1E90130BD
:1090A0009860D1E9010358605068884201D188680E
:1090B0005060002008611068401E10601068704702
:1090C000034B0360034B0B60802313607047000069
:1090D000A80E0020FC0E002000F1080141604FF0B6
:1090E000FF31816000F10801C16001610021016070
:1090F000704700210161704710B502460B685C1C87
:109100000CB9106907E002F1080000E0406844680B
:1091100024689C42FAD944684C604C68A16088601D
:1091200041600A611468641C146010BD42684A60A2
:1091300093688B60936859609160086103685B1C59
:109140000360704700BF502080F31188BFF34F8F3A
:10915000BFF36F8F00BF0E480068401C0C490860C9
:1091600008460068012812D10A480068C0B208B950
:10917000012000E0002050B900BF502080F311888A
:10918000BFF34F8FBFF36F8F00BF00BFFEE7704785
:10919000FC01002004ED00E00D48006850B900BF5C
:1091A000502080F31188BFF34F8FBFF36F8F00BF44
:1091B00000BFFEE706480068401E054908600846F3
:1091C000006820B9002080F3118800BF00BF7047FD
:1091D000FC01002070B506463546002E3FD0083D04
:1091E0002C461F4960680968084008B1012000E06A
:1091F000002050B900BF502080F31188BFF34F8F7B
:10920000BFF36F8F00BF00BFFEE7206808B90120E1
:1092100000E0002050B900BF502080F31188BFF358
:109220004F8FBFF36F8F00BF00BFFEE70C49606830
:109230000968084098B1206888B9094960680968D8
:109240008843606000F0AAF806496068096808442D
:10925000044908602046FFF7B5FC00F045FB70BDEF
:10926000F8010020F001002000204FF0E02108610B
:109270008861064800684FF47A71B0FBF1F0401E37
:109280004FF0E0214861072008617047A4010020E9
:1092900070B504460025D4B11248006808B9012011
:1092A00000E0002050B900BF502080F31188BFF3C8
:1092B0004F8FBFF36F8F00BF00BFFEE700F06EF867
:1092C00000212046FFF7B0FA00F00EFB05463DB93D
:1092D0004FF0805004490860BFF34F8FBFF36F8F8A
:1092E00070BD0000E001002004ED00E010B586B084
:1092F00000200590049003AA04A905A8FFF7E0FE4A
:109300000022DDE904101346CDE9002102901CA1E2
:109310001D48039A00F0E8F91C49086008460068F7
:1093200008B1012400E00024012C15D100BF502019
:1093300080F31188BFF34F8FBFF36F8F00BF4FF0E3
:10934000FF301349086001201249086000201249CB
:10935000086000F01BF910E0601C08B1012000E07B
:10936000002050B900BF502080F31188BFF34F8F09
:10937000BFF36F8F00BF00BFFEE706B010BD000057
:1093800049444C4500000000898A0008DC010020A7
:10939000D8010020C4010020BC0100200248006860
:1093A000401C014908607047E00100201D4800682A
:1093B00018B101201C49086032E000201A490860F9
:1093C0001A480068B0FA80F0C0F11F0101EB81007B
:1093D000174A52F8200008B1012000E0002050B9DF
:1093E00000BF502080F31188BFF34F8FBFF36F8F02
:1093F00000BF00BFFEE701EB81020D4B03EB8200D3
:1094000042685268426000F108024368934202D108
:109410004268526842604268D268064B1A6000BFD8
:1094200070470000E0010020CC010020C0010020B6
:10943000581A0020A801002007B582B0012010238F
:10944000374A082100900420FBF7BBFB01201223C0
:1094500000220C2100903720FBF7A0FA01201223F4
:1094600002460C2100904B20FBF798FA01201223B2
:109470000222282100903720FBF790FA01201223C6
:109480000322282100904B20FBF788FA9DF8090061
:10949000012808D100201023224A0C2100905D20D1
:1094A000FBF78FFB07E0002010231E4A28210090C5
:1094B0005D20FBF786FB9DF80800082808D10120F5
:1094C000102319A21E2100900F20FBF77AFB25E044
:1094D0009DF80800092808D10120102313A21E219D
:1094E00000900F20FBF76DFB18E09DF808000A289C
:1094F00008D1012010230EA21E2100900F20FBF79F
:1095000060FB0BE09DF808000B2807D10120102319
:1095100008A21E2100900F20FBF753FB05B000BDF1
:1095200029010020000100204C3100004C320000D5
:109530004C3300004C3400001148007800B97047EB
:109540000F480078662818D10D484078A8B90C4813
:109550008078012808D10A48C07A0A49087008486A
:10956000007B0949087008E005488078032803D18A
:109570000348C078012800D000BF00BFDFE700002B
:10958000A80A00207E0100207F0100201CB5384978
:10959000084600780190FF200A46107008460078BF
:1095A00000909DF8000000F0F0009DF8002090422F
:1095B00001D1012000E0002050B900BF502080F30D
:1095C0001188BFF34F8FBFF36F8F00BF00BFFEE75F
:1095D0009DF8000000F05000264A10700720264A2F
:1095E000106009E024480068401E234A10609DF87E
:1095F00000004006000E00909DF8000000F0800082
:109600008028EFD01C480068C0F10700042801D171
:10961000012000E0002050B900BF502080F31188E5
:10962000BFF34F8FBFF36F8F00BF00BFFEE712483D
:1096300000680002104A10601046008800F4E060E4
:1096400010600B4A019810700C48006840F47000DC
:109650000A4908600846006840F070400860FFF75B
:1096600003FE002006490860F6F780FD00201CBDBF
:1096700000E400E0000200200402002020ED00E0F1
:10968000FC0100202DE9FF4F85B080468946174632
:10969000DDE912ABB800FFF703FB064656B15420D4
:1096A000FFF7FEFA04460CB1266304E03046FFF7EC
:1096B00091FD00E000248CB1002084F85100CDE938
:1096C00000ABCDE902403A4649464046089BFFF7C9
:1096D000EFF92046FFF7F4F8012501E04FF0FF35E0
:1096E000284609B0BDE8F08F2DE9F04F85B0074658
:1096F000884691469A46DDE90EB6109C0EB10120CF
:1097000000E0002050B900BF502080F31188BFF363
:109710004F8FBFF36F8F00BF00BFFEE70CB101207A
:1097200000E0002050B900BF502080F31188BFF343
:109730004F8FBFF36F8F00BF00BFFEE75420039031
:109740000398542801D1012000E0002050B900BF47
:10975000502080F31188BFF34F8FBFF36F8F00BF8E
:1097600000BFFEE7B4B1AEB125462C462E63022001
:1097700085F85100002004A953464A46CDE900B1BE
:10978000CDE9025041463846FFF792F92846FFF7E7
:1097900097F801E000200490049805B0BDE8F08F30
:1097A0002DE9F0414FF0000844480068002877D1C7
:1097B00043480068451C4248056015BB41480068A5
:1097C000006808B9012000E0002050B900BF502017
:1097D00080F31188BFF34F8FBFF36F8F00BF00BFBF
:1097E000FEE7384807683848006836490860364858
:1097F000076036480068401C34490860FFF716FAD5
:1098000000BF3348006885423CD300BF2D48006844
:10981000006808B9012000E0002020B14FF0FF30BF
:109820002B4908602DE027480068C068C468666856
:10983000B54202D22648066023E0201DFFF72CFC2B
:10984000A06A18B104F11800FFF726FC94F82C1058
:10985000012088401F49096808431E490860E16AE1
:1098600001EB81011C4A02EB8100211DFFF75EFC28
:109870001A49E06A0968C96A8842C7D34FF00108EB
:10988000C4E700BF15480068C06A00EB80001249B9
:1098900051F82000012801D94FF0010805E0FFE749
:1098A0000F480068401C0E4908600E48006808B167
:1098B0004FF001084046BDE8F0810000E0010020C3
:1098C000BC010020AC010020B0010020D00100202C
:1098D000D8010020C0010020581A0020A801002053
:1098E000C8010020CC01002070B5002400263648B5
:1098F000006850B900BF502080F31188BFF34F8F2C
:10990000BFF36F8F00BF00BFFEE7FFF71BFC2E48C1
:109910000068401E2C4908600846006800284FD1A6
:109920002A48006800284BD024E02948C068C46851
:1099300004F11800FFF7B0FB201DFFF7ADFB94F812
:109940002C100120884023490968084321490860F8
:10995000E16A01EB8101204A02EB8100211DFFF742
:10996000E5FB1E49E06A0968C96A884202D3012002
:109970001B4908601648006808B9012000E0002073
:109980000028D2D00CB1FFF751F91648056865B12F
:1099900000BFFFF705FF10B10120114908606D1EDF
:1099A000002DF6D100200F4908600D48006838B13D
:1099B000012630070C490860BFF34F8FBFF36F8F4C
:1099C000FFF7EAFB304670BDE0010020B80100203F
:1099D0000C1B0020C0010020581A0020A801002004
:1099E000CC010020C801002004ED00E010B50246C3
:1099F0001378012002E0145C6340401C8842FADBCB
:109A0000184610BD0000000000000000002F0000FC
:109A100000000700070000147F147F1400242A7F31
:109A20002A120062640813230036495522500000B0
:109A30000503000000001C224100000041221C0020
:109A40000014083E08140008083E0808000000A0A2
:109A5000600000080808080800006060000000209E
:109A600010080402003E5149453E0000427F40007C
:109A7000004261514946002141454B310018141202
:109A80007F10002745454539003C4A4949300001CF
:109A90007109050300364949493600064949291E1E
:109AA0000000363600000000563600000008142280
:109AB0004100001414141414000041221408000280
:109AC0000151090600324959513E007C1211127CA5
:109AD000007F49494936003E41414122007F4141D2
:109AE000221C007F49494941007F09090901003EC4
:109AF0004149497A007F0808087F0000417F410002
:109B0000002040413F01007F08142241007F404077
:109B10004040007F020C027F007F0408107F003E5F
:109B20004141413E007F09090906003E4151215E45
:109B3000007F091929460046494949310001017F42
:109B40000101003F4040403F001F2040201F003FD8
:109B50004038403F0063140814630007087008078A
:109B600000615149454300007F41410000552A559D
:109B70002A55000041417F00000402010204004018
:109B8000404040400000010204000020545454783A
:109B9000007F48444438003844444420003844445A
:109BA000487F00385454541800087E0901020018F8
:109BB000A4A4A47C007F080404780000447D400035
:109BC000004080847D00007F102844000000417F19
:109BD0004000007C04180478007C080404780038F5
:109BE0004444443800FC242424180018242418FC7D
:109BF000007C0804040800485454542000043F44E6
:109C00004020003C4040207C001C2040201C003CA8
:109C10004030403C004428102844001CA0A0A07CF8
:109C2000004464544C441414141414140000000030
:109C300000000000000000000000FC000000000028
:109C400002000000000C020C0200000000000000F6
:109C500090D0BCD0BC900003000300001824FE4448
:109C60008C000302070201001824D8B04C800003C6
:109C700000010201C038E438E000010202010202E2
:109C8000080600000000000000000000000000F8CE
:109C90000402000000010204000204F800000004B5
:109CA000020100009060F8609000000001000000D8
:109CB0002020FC2020000000010000000000000027
:109CC00000000806000000002020202020000000E6
:109CD0000000000000000000000000020000000082
:109CE0000080601C0200040300000000F80404046B
:109CF000F8000102020201000008FC00000000025E
:109D00000302000018844424180003020202020027
:109D100008042424D80001020202010040B088FC9B
:109D200080000000000302003C242424C40001023F
:109D300002020100F824242CC000010202020100EA
:109D40000C04E41C0400000003000000D8242424B8
:109D5000D80001020202010038444444F800000324
:109D600002020100000010000000000002000000DC
:109D700000002000000000000600000000205088C5
:109D800004020000000001029090909090000000FA
:109D900000000000000204885020000201000000C2
:109DA0001804C4241800000002000000F804E49421
:109DB000F80001020202020000E09CF080000203B1
:109DC0000000030204FC2424D80002030202010064
:109DD000F80404040C0001020202010004FC040463
:109DE000F80002030202010004FC24740C000203C8
:109DF0000202030004FC24740C00020302000000B1
:109E0000F0080444CC4000010202010004FC2020C0
:109E1000FC040203000003020404FC040400020228
:109E200003020200000404FC04040604040300000E
:109E300004FC24D00C0402030200030204FC04000E
:109E40000000020302020203FC3CC03CFC000300D1
:109E50000300030004FC30C4FC04020302000300FE
:109E6000F8040404F80001020202010004FC2424A6
:109E70001800020302000000F8848404F8000102C4
:109E80000207050004FC2464980002030200030298
:109E9000182424448C000302020201000C04FC0478
:109EA0000C0000020302000004FC0000FC0400019E
:109EB00002020100047C80E01C040000030000009A
:109EC0001CE03CE01C00000300030000049C609CBC
:109ED0000400020300030200041CE01C0400000252
:109EE000030200000C84641C04000203020203004D
:109EF0000000FE020200000007040400000E30C053
:109F00000000000000010200000202FE0000000448
:109F1000040700000004020400000000000000002C
:109F200000000000000008080808080800000200FF
:109F300000000000000000000040A0A0C0000001E0
:109F40000202030204FC2020C00000030202010000
:109F500000C02020600000010202020000C0202496
:109F6000FC0000010202030200C0A0A0C00000012A
:109F7000020202000020F82424040002030202006E
:109F80000040A0A0602000070A0A0A0404FC202068
:109F9000C0000203020003020020E40000000002EF
:109FA00003020000000020E4000008080807000089
:109FB00004FC80E020200203020003020404FC00F1
:109FC0000000020203020200E020E020C0000300C3
:109FD0000300030020E02020C0000203020003026F
:109FE00000C02020C00000010202010020E020206B
:109FF000C000080F0A02010000C02020E00000019C
:10A00000020A0F0820E040202000020302000000A6
:10A010000060A0A020000002020203000020F8203F
:10A02000000000000102020020E00020E00000012A
:10A030000202030220E020806020000003010000F3
:10A040006080E0806000000300030000206080600A
:10A05000200002030003020020E0208060200808A6
:10A06000070100000020A06020000002030202009F
:10A07000000020DE0200000000070400000000FFD6
:10A0800000000000000F00000002DE2000000004BD
:10A0900007000000020102040402000000000000AA
:10A0A00000000000000000000000000000000000B0
:10A0B000000000F800000000000000333000000045
:10A0C00000100C06100C060000000000000000004C
:10A0D00040C07840C0784000043F04043F040400BE
:10A0E000007088FC08300000001820FF211E0000CE
:10A0F000F008F000E018000000211C031E211E00E3
:10A1000000F00888700000001E2123241927211068
:10A1100010160E000000000000000000000000000B
:10A12000000000E0180402000000000718204000B2
:10A1300000020418E00000000040201807000000A2
:10A14000404080F0804040000202010F0102020006
:10A15000000000F0000000000101011F01010100EA
:10A16000000000000000000080B07000000000004F
:10A1700000000000000000000001010101010101D8
:10A18000000000000000000000303000000000006F
:10A190000000000080601804006018060100000044
:10A1A00000E010080810E000000F102020100F0041
:10A1B000001010F8000000000020203F20200000C8
:10A1C0000070080808887000003028242221300020
:10A1D00000300888884830000018202020110E0028
:10A1E0000000C02010F8000000070424243F2400D1
:10A1F00000F80888880808000019212020110E00A6
:10A2000000E0108888180000000F112020110E00B7
:10A2100000380808C83808000000003F00000000AF
:10A220000070880808887000001C222121221C0070
:10A2300000E010080810E0000000312222110F0099
:10A24000000000C0C000000000000030300000002E
:10A25000000000800000000000008060000000009E
:10A2600000008040201008000001020408102000B7
:10A270004040404040404000040404040404040002
:10A280000008102040800000002010080402010097
:10A29000007048080808F000000000303601000097
:10A2A000C030C828E810E0000718272423140B004A
:10A2B0000000C038E0000000203C230202273820C4
:10A2C00008F8888888700000203F202020110E00A8
:10A2D000C03008080808380007182020201008009F
:10A2E00008F808080810E000203F202020100F0088
:10A2F00008F88888E8081000203F20202320180054
:10A3000008F88888E8081000203F200003000000BB
:10A31000C03008080838000007182020221E02005C
:10A3200008F808000008F808203F210101213F201B
:10A33000000808F8080800000020203F2020000046
:10A3400000000808F8080800C08080807F00000036
:10A3500008F888C028180800203F2001263820006F
:10A3600008F8080000000000203F202020203000D6
:10A3700008F8F800F8F80800203F003F003F2000F0
:10A3800008F830C00008F808203F200007183F00F8
:10A39000E01008080810E0000F10202020100F0027
:10A3A00008F808080808F000203F2101010100001A
:10A3B000E01008080810E0000F18242438504F005F
:10A3C00008F8888888887000203F2000030C30201F
:10A3D00000708808080838000038202121221C005D
:10A3E000180808F8080818000000203F20000000A6
:10A3F00008F808000008F808001F202020201F008F
:10A400000878880000C83808000007380E010000EE
:10A41000F80800F80008F800033C0700073C0300B8
:10A42000081868808068180820302C03032C30201E
:10A430000838C800C83808000000203F200000008D
:10A4400010080808C83808002038262120201800E5
:10A45000000000FE020202000000007F40404000B9
:10A46000000C30C000000000000000010638C000F1
:10A4700000020202FE000000004040407F00000099
:10A4800000000402020204000000000000000000BE
:10A4900000000000000000008080808080808080BC
:10A4A00000020204000000000000000000000000A4
:10A4B00000008080808000000019242222223F209A
:10A4C00008F8008080000000003F112020110E00DD
:10A4D0000000008080800000000E1120202011006C
:10A4E000000000808088F800000E112020103F201E
:10A4F0000000808080800000001F222222221300A2
:10A50000008080F0888888180020203F20200000EC
:10A510000000808080808000006B949494936000A1
:10A5200008F8008080800000203F210000203F20AC
:10A5300000809898000000000020203F20200000AC
:10A54000000000809898000000C08080807F00009C
:10A5500008F8000080808000203F24022D30200079
:10A56000000808F8000000000020203F2020000024
:10A570008080808080808000203F20003F20003F3E
:10A580008080008080800000203F210000203F204C
:10A590000000808080800000001F202020201F00FD
:10A5A000808000808000000080FFA12020110E002C
:10A5B0000000008080808000000E112020A0FF801D
:10A5C000808080008080800020203F2120000100CA
:10A5D000000080808080800000332424242419001F
:10A5E000008080E0808000000000001F202000002C
:10A5F0008080000000808000001F202020103F206D
:10A60000808080000080808000010E3008060100FC
:10A6100080800080008080800F300C030C300F00A1
:10A6200000808000808080000020312E0E312000CC
:10A63000808080000080808080818E7018060100FC
:10A6400000808080808080000021302C222130001A
:10A6500000000000807C020200000000003F40403B
:10A6600000000000FF00000000000000FF000000EC
:10A670000002027C800000000040403F000000001B
:10A6800000060101020204040000000000000000B6
:10A6900000000000000000000000000000000000BA
:10A6A00000000000000000000000000000000000AA
:10A6B000000000000000000000F0F0F000000000CA
:10A6C0000000000000017F01000000000000000009
:10A6D000001C1C1C0000000000008060301C8C600E
:10A6E000301C0C0000000000000000000000000012
:10A6F000000000000000000000000000000000E07A
:10A700000000000000E000000086E69F8686868646
:10A71000E69F860000011F01010101011F010100E8
:10A72000000080C06020F820E0C0000000000307A7
:10A730000C18FF70E18100000000070F10107F105F
:10A740000F0700008060206080000000E020000013
:10A750000F3020309F70DC371030C0000000100E2A
:10A7600003000718101807000000C02020E0C000F8
:10A770000000000080E01F38E88703C43C040000AC
:10A78000070F1810100B070D1010080000808C4CDC
:10A790003800000000000000000000000000000081
:10A7A00000000000000000000000000000000000A9
:10A7B00000000000000080E03008040000000000FD
:10A7C00000FEFF0100000000000000000000030F79
:10A7D0001820400000040830E08000000000000065
:10A7E0000000000001FFFE000000000000402018F3
:10A7F0000F03000000000000000000000000C00087
:10A8000000000000004266663C18FF183C66664285
:10A810000000000000000300000000000000000035
:10A820000000800000000000001010101010FF1049
:10A8300010101010000000000000030000000000D5
:10A840000000000000000000000000000000000008
:10A85000000000000000000000808C4C3800000068
:10A8600000000000000000000000000000000000E8
:10A870000010101010101010101010000000000038
:10A8800000000000000000000000000000000000C8
:10A8900000000000000000000000000000000000B8
:10A8A00000001C1C1C000000000000000000000054
:10A8B00000000000E0380C000000000080701C0365
:10A8C000000000000060380E0100000000000000E1
:10A8D000000080C060202060C080000000FEFF01FA
:10A8E0000000000001FFFE000001070E1810101804
:10A8F0000E0701000000808080C0E0000000000022
:10A900000000000000FFFF00000000000000101029
:10A91000101F1F1010100000008040202020206019
:10A92000C080000000030300804020381F070000A3
:10A93000001C1A1918181818181F00000080C020D1
:10A94000202060C080000000000303001010182FBA
:10A95000E780000000070F10101010180F0700000C
:10A96000000000000000C0E0F000000000C0B0885F
:10A97000868180FFFF808000000000000010101F13
:10A980001F1010000000E060606060606060000008
:10A9900000003F1008080818F0E0000000070B1046
:10A9A0001010101C0F030000000080C04020202069
:10A9B000E0C0000000FCFF211008080818F0E000CB
:10A9C0000001070C18101010080F03000000C0E071
:10A9D0006060606060E06000000003000000E0185C
:10A9E0000700000000000000001F1F000000000022
:10A9F0000080C0602020202060C080000087EF2CF5
:10AA00001818303068CF830000070F08101010109E
:10AA1000180F07000000C0C020202020C0800000C8
:10AA2000001F3F604040402010FFFE0000000C1C53
:10AA3000101010080F0300000000000000000000CC
:10AA40000000000000000000000E0E0E00000000DC
:10AA500000000000001C1C1C0000000000000000A2
:10AA6000000000000000000000000000000C0C00CE
:10AA70000000000000000000005838000000000046
:10AA8000000000000000008040201000000010289E
:10AA900044820100000000000000000000000102EC
:10AAA000040810000000000000000000000000008A
:10AAB000008484848484848484848400000000006E
:10AAC0000000000000000000000010204080000096
:10AAD0000000000000000000000001824428100077
:10AAE00000001008040201000000000000C0202047
:10AAF0001010101030E0C0000003030000F0100838
:10AB00000C070300000000001C1C1C0000000000DB
:10AB1000000000C0406020202040C00000FCFF0179
:10AB2000F00E03C1FE03807F0001070E0811111013
:10AB3000110904020000000080E0E00000000000B5
:10AB40000000807C4340477FF880000010181F10F1
:10AB500000000000131F1C1020E0E02020202060D7
:10AB6000C080000000FFFF10101010182FE78000B9
:10AB7000101F1F1010101010180F0700000080C0C9
:10AB8000402020202060E00000FCFF0100000000C9
:10AB9000000001000001070E181010100804030047
:10ABA00020E0E02020202040C080000000FFFF00C7
:10ABB0000000000001FFFE00101F1F1010101808F9
:10ABC0000E07010020E0E0202020202020608000EF
:10ABD00000FFFF101010107C00000000101F1F105D
:10ABE000101010101018060020E0E0202020202077
:10ABF0006060800000FFFF101010107C000001005A
:10AC0000101F1F100000000000000000000080C0A6
:10AC10006020202040E0000000FCFF0100004040D8
:10AC2000C0C140400001070E181010100F0F0000A7
:10AC300020E0E0200000000020E0E02000FFFF1006
:10AC40001010101010FFFF00101F1F100000000058
:10AC5000101F1F100000202020E0E0202020000016
:10AC60000000000000FFFF000000000000001010C6
:10AC7000101F1F101010000000000000202020E016
:10AC8000E020202000000000000000FFFF00000086
:10AC90000060E0808080C07F3F00000020E0E02076
:10ACA000000020A06020200000FFFF30187CE3C0DF
:10ACB00000000000101F1F10000001131F1C1810BF
:10ACC00020E0E020000000000000000000FFFF0086
:10ACD0000000000000000000101F1F1010101010D6
:10ACE0001018060020E0E0E000000000E0E0E020B6
:10ACF00000FF013FFEC0E01E01FFFF00101F10001B
:10AD0000031F0300101F1F1020E0E0C00000000020
:10AD10000020E02000FF0003071C78E08000FF0017
:10AD2000101F100000000000030F1F00000080C073
:10AD300060202060C080000000FEFF0100000000D5
:10AD400000FFFE000001070E181010180C0701008C
:10AD500020E0E0202020202060C0800000FFFF20B5
:10AD600020202020301F0F00101F1F1000000000A7
:10AD700000000000000080C060202060C080000053
:10AD800000FEFF010000000000FFFE000001070EB2
:10AD90001111133C7C67210020E0E02020202020BE
:10ADA00060C0800000FFFF101030F0D0080F0700D7
:10ADB000101F1F10000000030F1C10100080C06047
:10ADC000202020204040E00000070F0C18183030F1
:10ADD00060E08100001F0C0810101010180F070011
:10ADE0008060202020E0E020202060800100000022
:10ADF00000FFFF000000000100000000101F1F10F6
:10AE00000000000020E0E020000000000020E02022
:10AE100000FFFF00000000000000FF0000070F1807
:10AE200010101010100807002060E0E02000000063
:10AE300020E060200000077FF88000807C03000095
:10AE400000000000071F1C070000000020E0E020B9
:10AE500000E0E0200020E0200007FFF8E01FFFFCFA
:10AE6000E01F00000000031F0300011F030000009B
:10AE7000002060E0A0000020E0602000000000034F
:10AE80008F7CF8C6010000000010181E1300011787
:10AE90001F1810002060E0E02000000020E060208B
:10AEA000000001073EF8E018070000000000001055
:10AEB000101F1F101000000000806020202020A024
:10AEC000E0E0200000000000C0F03E0F03000000A2
:10AED00000101C1F171010101018060000000000B2
:10AEE00000FC0404040404000000000000FF000053
:10AEF0000000000000000000007F40404040400093
:10AF0000000010E000000000000000000000000051
:10AF1000031C60800000000000000000000000032F
:10AF20000C70800000000404040404FC0000000015
:10AF300000000000000000FF000000000000404092
:10AF40004040407F0000000000000010080C040C8E
:10AF500008100000000000000000000000000000D9
:10AF600000000000000000000000000000000000E1
:10AF700000000000000000000000000000000000D1
:10AF800000000000808080808080808080808080C1
:10AF90000000000404080800000000000000000099
:10AFA00000000000000000000000000000000000A1
:10AFB0000000000000000000000000000000000091
:10AFC000000098D844642424FCF80000000F1F18E7
:10AFD000101010081F1F10180020E0F000000000E3
:10AFE000000000000000FFFF180804040CF8F00047
:10AFF00000001F0F18101010180F030000000000B1
:10B00000000000000000000000E0F8180404043C08
:10B010003800000000030F0C10101010080600008C
:10B020000000000000000020E0F0000000E0F81C3C
:10B0300004040408FFFF000000030F18101010089C
:10B040001F0F0800000000000000000000000000CA
:10B050000000E0F8484444444C7870000000030FBE
:10B060000C181010100804000000000080C06020C0
:10B0700020E0C00000040404FFFF040404040000F6
:10B08000000010101F1F1010100000000000000032
:10B090000000000000000000000070F88C04048C28
:10B0A000F874040C007076CF8D8D8D89C87870008F
:10B0B0000020E0F000000000000000000000FFFFA2
:10B0C00008040404FCF8000000101F1F100000100A
:10B0D0001F1F100000000000006060000000000062
:10B0E0000000040404FCFC0000000000000010103C
:10B0F000101F1F1010100000000000000000006072
:10B100006000000000000000040404FCFC000000DB
:10B110000000C0C08080C07F3F0000000020E0F041
:10B1200000000000000000000000FFFF80C0F41CD1
:10B130000404000000101F1F1100031F1C1010004A
:10B140000000202020E0F0000000000000000000CF
:10B1500000FFFF000000000000001010101F1F1073
:10B1600010100000000000000000000000000000BF
:10B1700004FCFC0804FCFC0804FCFC00101F1F106D
:10B18000001F1F10001F1F10000000000000000023
:10B19000000000000004FCFC08080404FCF80000A7
:10B1A00000101F1F100000101F1F100000000000E3
:10B1B000000000000000000000E0F0180C04040C87
:10B1C00018F0E00000030F0C101010100C0F03001B
:10B1D0000000000000000000000000000004FCFC73
:10B1E000080404040CF8F0000080FFFF88901010A1
:10B1F0001C0F030000000000000000000000000021
:10B2000000E0F81C04040408F8FC000000030F1818
:10B2100010109088FFFF8000000000000000000078
:10B2200000000000040404FCFC100804040C0C00E2
:10B230001010101F1F101010000000000000000070
:10B24000000000000000000000003078CCC48484BE
:10B25000840C1C0000001E1810101011190F06009D
:10B260000000000000C00000000000000004040412
:10B27000FFFF040404000000000000000F1F101076
:10B28000100C0000000000000000000000000000A2
:10B290000004FCFE00000004FCFE000000000F1F84
:10B2A000181010081F0F0800000000000000000028
:10B2B0000000000000040C3CFCC40000C43C0C0472
:10B2C00000000000010F1E0E010000000000000041
:10B2D0000000000000000000043CFCC400E47CFC12
:10B2E00084807C040000071F070000071F07000080
:10B2F0000000000000000000000000000004041C2A
:10B300007CE4C0341C0404000010101C1601131F40
:10B310001C181000000000000000000000000000E9
:10B3200000040C3CFCC400C43C0404000000C080C9
:10B33000C1370E0100000000000000000000000006
:10B340000000000000001C0404C4F47C1C04000085
:10B350000000101C1F17111010180E000000000034
:10B36000000000F80C04000000000000001028EFAE
:10B3700000000000000000000000003F60400000EE
:10B38000000000000000FF000000000000000000BE
:10B390000000FF0000000000000000000000FF00AF
:10B3A000000000000000040CF80000000000000095
:10B3B00000000000EF2810000000000000004060C6
:10B3C0003F00000000000000001806020204081000
:10B3D00020203008000000000000000000000000F5
:10B3E0000000000000000000000000000000F0105D
:10B3F000101010FF10101010F000000000000F04DB
:10B40000040404FF040404040F0000004040405FF3
:10B41000555555755555555F404040000040200F2B
:10B42000094989790909090F2040000000FE0242FC
:10B430004ACA4A4ACA4A4A4202FE000000FF405035
:10B440004C4340404F50505C40FF00000000F888E3
:10B45000888888FF88888888F800000000001F0816
:10B460000808087F888888889F80F0008082828210
:10B47000828282E2A2928A8682808000000000009E
:10B480000040807F0000000000000000101010FF4E
:10B49000109008888888FF88888808000444827F84
:10B4A00001808040432C102846818000001010103D
:10B4B00010D030FF30D0121C101000001008040211
:10B4C000010000FF000001020408100004040484CD
:10B4D000E43C2724242424E404040400040201009E
:10B4E000FF0909090949897F0000000000FE225A6E
:10B4F0008600FE9292929292FE00000000FF0408E5
:10B500000700FF4020030C1422414000008040202F
:10B5100018068000071820408000000001002070FD
:10B5200028262120202438600001010000101292FA
:10B530009292929292121202FE0000000000003FCE
:10B54000101010103F0040807F0000008082828237
:10B55000FE8282828282FE8282828000008040306F
:10B560000F0000000000FF000000000000001011AC
:10B57000161010F0101014131000000081814141CA
:10B5800021110D030D1121414181810000084888DE
:10B5900008C83800901010FF101010000020100C88
:10B5A000030418000043807F0000000020102CE7F7
:10B5B000242400E22C20BF2028E600000101017FA6
:10B5C0002111804F20100F10204F8000008060F864
:10B5D0000740300FF888888888080800010000FFBD
:10B5E00000000000FF080808080800000010608044
:10B5F00000FF000000FF0000C0300000404040435A
:10B60000407F4040407F4241404040001010F19652
:10B61000909010E80784FC8444C4040080601F40BC
:10B62000807F013F41405F44484778002010EC276D
:10B63000F42CE00022920ED2221E000080601F092E
:10B640003F89FF000A0909FF0909080040484848E6
:10B650007F48484800901010FF10100040C4444438
:10B660003F242424000043807F000000404042CC5F
:10B670000040A09E8282829EA02020000000003F09
:10B68000908840432C10284641808000809090484C
:10B690004C57242424544C4480808000000000FF38
:10B6A0004949497F494949FF000000001010FF1037
:10B6B00090E02F29E909E9292FE0000042827F412B
:10B6C0004425150D05FE0D1525454400008060F844
:10B6D0000740300FF888888888080800010000FFBC
:10B6E00000000000FF08080808080000404424A4E7
:10B6F000948C84FF848C94A4244440004040405F98
:10B700004A4A4A4A4A4A4A5F4040400020222A2A7E
:10B71000AA6A3A2E29292929292020000804020191
:10B72000FF555555555555FF0000000000083000E5
:10B73000FF20202020FF2020222C200004040201D2
:10B74000FF8040300E0106182040800000048484F1
:10B750004424548F1424448484040000413900009C
:10B760003C4040424C404070040931002038E730F2
:10B77000004848FF484800FE42B20E00222712123D
:10B780000082621F020200FF08100F00100C4444E8
:10B79000444445C64444444444140C008040201EA4
:10B7A0002040407F4444444444404000000000C0E6
:10B7B00080808080808080FC84808080808080C0C9
:10B7C000C0000000000000FF7F404040404040FFBC
:10B7D00040404040404040FF7F000000000000002B
:10B7E000000000000000007F70000000000000006A
:10B7F0000000000000000000000000000000000049
:10B80000000000FCF8000000000000000000000044
:10B810000000000000000000FFFE0202020202021F
:10B82000020202FFFF020202020202020202FF0300
:10B8300000000000000000001F1F040404040404B2
:10B84000040404FFFF0404040404040404041F00AB
:10B8500000000000000000000000000000000000E8
:10B860000000007F3F00000000000000000000001A
:10B8700000000000000000000000000000000000C8
:10B8800000000000000000000000000000000000B8
:10B8900000F8F8F0F0702000000000000000000048
:10B8A0000000000000000000000000000000000098
:10B8B0000000000000000000000000008000000008
:10B8C0000000000000000000000000000000000078
:10B8D00000FFFFFFFF00000000000000000000006C
:10B8E0000000000000000000808000000000000058
:10B8F00000000000000000000000000000FFFFFE4C
:10B9000006060606060606060606060606060606D7
:10B9100006FFFFFFFF0606060606060606060606E3
:10B9200006060606060606FFFFFFFF0702000000E8
:10B9300000000000000000000000000000FFFFFF0A
:10B9400000000000000000000000000000000000F7
:10B9500000FFFFFFFF0000000000000000000000EB
:10B9600000000000000000FFFFFFFF0000000000DB
:10B9700000000000000000000000000000FFFFFFCA
:10B980001818181818181818181818181818181837
:10B9900018FFFFFFFF18181818181818181818188B
:10B9A00018181818181818FFFFFFFF0000000000F3
:10B9B0000000000000000000000000000201010083
:10B9C0000000000000000000000000000000000077
:10B9D00000FFFFFFFF00000000000000000000006B
:10B9E0000000000000000001010000000000000055
:10B9F0000000000000000000000000000000000047
:10BA00000000000000000000000000000000000036
:10BA100000FFFFFFFF00000000000000000000002A
:10BA20000000000000000000000000000000000016
:10BA30000000000000000000000000000000000006
:10BA400000000000000000000000000000000000F6
:10BA5000001F1F0F0F00000000000000000000008A
:10BA600000000000000000000000000000000000D6
:10BA70000000000042F22EE200F453F25A56F000A9
:10BA8000000702070807010701090F001011F20063
:10BA90000000C03FC00000000000070209060100CE
:10BAA000010608001011F200FE0A2A4A89493900ED
:10BAB0000804030609080A0908090A0000FE020230
:10BAC000F29292F20202FE00000F04040404040445
:10BAD00004040F0094F39200F21410DF1014F2002B
:10BAE000000F0408090402010204090000001010FC
:10BAF000F8000000000040407F400000000000000F
:10BB000000000000007008080810E00000605844C1
:10BB100042417000000000000000000000300808F2
:10BB200008F060000030404141221C00000000008D
:10BB3000000000000000804030F8000000060948C6
:10BB4000487F4000000000000000000004FD26E4E3
:10BB500044F342FE2212F2000807080F0007080B08
:10BB600008090D00202424BF2424488808FF080069
:10BB70000809090705050009080F000008F453FA31
:10BB800056F0896741E94F0008070107090F0002D5
:10BB9000020F020002020202FE0212224282020090
:10BBA000000000000F000000000100004040404085
:10BBB00040404040404040000000000000000000C5
:10BBC0000000000010FC03086888090A08E8080063
:10BBD000000F0008080B080C0B080800DCB30880F5
:10BBE000FE2AEA2BEA2AEE00040402000F010701F4
:10BBF00007090F00645CF74410F7555555F710001E
:10BC000002020F0104070505050F02000024448409
:10BC1000641C00488808FF08080010080601030C8F
:10BC2000000021203F0000001028E7242400F21427
:10BC300010DF1014F20001013F110920271008073E
:10BC4000081027004020F807201807FC444444440B
:10BC5000040000003F000000003F0404040404004E
:10BC60000830C000FF000000FF00C03800002020A6
:10BC700021203F2020203F21202020002021E600FD
:10BC800040A09E8282829EA0200000001F082420E7
:10BC90001314081412212000002FA9A9AFA9F9A993
:10BCA000AFA9A92F000020203F2020203C202020E9
:10BCB0003F2020004444A4948C84BF848C94A444EA
:10BCC000440020202F2A2A2A2A2A2A2A2F2020002C
:10BCD00020222AAAEABAAEAAA9A9A9212000040210
:10BCE000013F2A2A2A2A2A2A3F000000041880FF3E
:10BCF000001010907F90121410000201003F2010DD
:10BD00000C0300030C1020008484444424548F143A
:10BD10002444448484002018001C2020222C20303D
:10BD2000000418004042CC008888FF888888FF887B
:10BD3000880020100F102028272020202F202000EE
:10BD40008844E2190020222222E222222000000060
:10BD50003F0000000020203F0000000008F8494A92
:10BD6000C81008E784FC44E40400201F00203F00C2
:10BD7000011F202F2427380008F493FA96F000D2F0
:10BD80008EE2929E0000201F041F243F0504043F02
:10BD900004040400202424BF242400488808FF0849
:10BDA00008001011110F0909000021203F000000B8
:10BDB0004048C4A6AB929292AAA6C240400000009E
:10BDC0003F2424243F2424243F00000090DCB39827
:10BDD0000424FF2400FE02629E00080804042111CE
:10BDE0000F01003F080807000C0424242425E62442
:10BDF000242424040C0020100F1020203F22222293
:10BE000022202000404141FF4141414141FF414149
:10BE1000400020100C0300000000003F0000000064
:10BE2000808888898E88F8888C8B8888800020207C
:10BE30001008040300030408102020000808FF88ED
:10BE40000070577505755770000021213F001212D0
:10BE50000A063F060A1212004020F807201807FCC5
:10BE600044444444040000003F000000003F040438
:10BE700004040400000008F18E88884828D80FF0D8
:10BE80002888888808000080704F80807F0202FF29
:10BE900081BF81889C83E00000000000000000005A
:10BEA000000000000000000000000000888888FFFB
:10BEB000888880A0202020FF2020200000C044444B
:10BEC000447F44242420018E80FF000000000000F5
:10BED0000000000000000000000000010000000061
:10BEE0000040F02C27F42CE06040E29CC262223E2D
:10BEF000000000807F05057F05FF080A0909FF098A
:10BF00000909080000000000000000010000000016
:10BF10000100000000000000888888FF888880A059
:10BF2000202020FF2020200000C04444447F4424DF
:10BF30002420018E80FF00000000000000000000AF
:10BF4000000000000000000100000000000010FFE1
:10BF50001090E0203EEA0A0AF22E20E00000008263
:10BF600082FF01804745351BFE0A172545C744005F
:10BF700000000001010000000000010000000000BE
:10BF8000000000008060FC0340201C0FF0888888BF
:10BF90008888000000010000FF0000000000FF088A
:10BFA0000808080800000000000001000000000070
:10BFB0000100000000000000000000F01010101050
:10BFC000101EFA10121CD09000000080601F21216A
:10BFD000413F8080433C3866C180E00000010000A2
:10BFE000000000010000000000000000010000004F
:10BFF000080808F00808082020FF202020E00000A2
:10C0000000003010100F088840201C038080807FC3
:10C01000000000000000000101000000000000011D
:10C0200001000000D0C00008055100080300000016
:10C030000000000080000000000000000000000080
:10C04000ACC00008F1500008030000000000000030
:10C05000800000000000000000000000C4C00008D4
:10C060003D510008030000000000000080000000B7
:10C070000000000000000000B8C00008495100089E
:10C08000030000000000000080000000000000002D
:10C090000000000000000000000000000102030496
:10C0A0000607080900000000010203044254344757
:10C0B0005461736B000000006C6F67696E666F54AB
:10C0C00061736B00746573745461736B00000000DE
:10C0D0005363616E4B65795461736B00FCC000085B
:10C0E000000000200C020000F0020008BCC10008A3
:10C0F0000C0200203C290000C05800084A80012D95
:10C10000FCFEFF87014707071F1E1CFF3718E422AC
:10C1100022F408390E113B0708013B090907620F99
:10C1200039384939580887FFFFFEFC80802E116797
:10C1300038E44040E43C5AFF3C193D593F0C190893
:10C14000080778E8080222F4C8E0E0E0782A0F0146
:10C1500089784CFEFF8F78AAFE782A3C783B38C05D
:10C1600001C978393F230F07100E445455207374CA
:10C17000617274202E2E2E143C2D2D13534E1C4C08
:10C180002031041A32041A33041234144D313A1B8C
:10C190004D32041A330413343A1A3C25123A1A4C1D
:10C1A00025192419235234055B6E756C6C321042CC
:0CC1B00001035524F41AAA01C10000008C
:0400000508000131BD
:00000001FF
